:100000000C9466000C9487000C9487000C94870075
:100010000C9487000C9487000C9487000C94870044
:100020000C9487000C9487000C9487000C94870034
:100030000C9487000C9487000C9487000C94870024
:100040000C9487000C9487000C9487000C94870014
:100050000C9487000C94390B0C9487000C94870047
:100060000C9487000C94E10D0C9487000C9487008D
:100070000C9487000C9487000C9487000C948700E4
:100080000C9487000C9487000C9487000C940F0C40
:100090000C94B7150C9487000C9487000C9487007F
:1000A0000C9487000C9487000C9487000C948700B4
:1000B0000C9487000C9487000C9487000C948700A4
:1000C0000C9487000C9487000C94870011241FBEA9
:1000D000CFEFD1E2DEBFCDBF00E00CBF14E0A0E067
:1000E000B2E0E8E6F3E800E00BBF02C007900D9233
:1000F000AC32B107D9F716E0ACE2B4E001C01D9212
:10010000AF3FB107E1F70E94B6030C94B2410C94E3
:100110000000109232048091320480933104809167
:100120003104809330048091300480932F04109226
:1001300033040895EEE6F0E080818260808383E0FE
:1001400084BD85BD8AEF87BD0895E1E7F0E0808139
:1001500081608083089580917100817008958091FD
:100160008404982F9295969596959370282F221F28
:100170002227221F9227282F22952F709227282F7F
:100180002695269592279170880F892B8093840459
:10019000089590937B0480937A0485EB9BE390937E
:1001A0008C0480938B0483E393E190939204809377
:1001B000910485E694ED90938804809387040895D4
:1001C00080917A0490917B04AC01440F452F441F29
:1001D000550B51954827592760918B0470918C04D9
:1001E00070937B0460937A048091910490919204BF
:1001F00090938C0480938B04209187043091880421
:100200003093920420939104C90100249695879518
:100210000794969587950794982F802D822793278A
:1002200084279527542F44275295550F507E8427B5
:1002300095279093880480938704660F771F6F5FDC
:100240007F4F869F9001879F300D969F300D112420
:10025000C9010895FC019081992351F08091C80053
:1002600085FFFCCF9093CE00319690819923B1F712
:1002700008951F93CF93DF93182F492FE0E1F7E202
:10028000C0E0D0E0812F942FBF010E9469419B0103
:100290006115710589F5812F942FBF010E94694175
:1002A000182F492FCF016AE070E00E946941FB01DD
:1002B0002196C430D10531F73097A1F18091C80063
:1002C00085FFFCCF812F942FBF010E946941605DA3
:1002D0006093CE00CF016AE070E00E9469419B010B
:1002E00061157105F9F0812F942FBF010E946941BA
:1002F000182F492FF901E2CF8091C80085FFFCCF6C
:10030000822F805D8093CE00812F942FBF010E94A9
:100310006941182F492FCF016AE070E00E946941BE
:10032000FB01CACFDF91CF911F910895982F9F7045
:100330009A3040F48091C80085FFFCCF905D909387
:10034000CE0008958091C80085FFFCCF995C909302
:10035000CE000895CF93DF93EC01892F99278295E2
:100360008F700097C1F48D2F9927009789F4CE01E3
:10037000929582958F7089279F708927009711F039
:100380000E9496018C2F0E949601DF91CF910895D3
:100390000E949601ECCF0E949601E5CF982F8091A4
:1003A000C80085FFFCCF9093CE0080E090E00895D8
:1003B0002091C800332727FD30952227330F221FB5
:1003C0003327C90108958091C80087FFFCCF809131
:1003D000CE0090E008959C018FEF80937F0493E01E
:1003E000283E390768F580937C0480937D04243689
:1003F0003105D8F0C90164E670E00E94694160935C
:100400007C04C9016AE070E00E946941CB016AE0A6
:1004100070E00E94694180937D04C9016AE070E048
:100420000E94694180937E0408952A30310548F77F
:10043000C9016AE070E00E94694180937E040895DA
:1004400010927C0410927D0410927E040895909185
:10045000340493609093340480933504089580911C
:1004600034048360809334040895F999FECF92BDDB
:1004700081BDF89A30B5F999FECF019692BD81BD44
:10048000F89A20B5932F80E030E0282B392BC90152
:100490000895F999FECF92BD81BDF89A80B508956F
:1004A000F999FECF92BD81BD60BDF894FA9AF99A90
:1004B00078940895FF920F931F938C01F62E672F67
:1004C0000E945002C80101966F2D0E9450021F9198
:1004D0000F91FF9008958091C90088618093C900B1
:1004E00083E38093CC001092CD008091C80087FDFB
:1004F0002FC08091C90080688093C9008091C1009D
:1005000088698093C1008FE18093C4001092C50078
:1005100090EC91B98CE382B987E384B995B99FEFE8
:1005200097B988EF8AB98BE08BB982E08DB99EB913
:1005300010BA91BB13BA94BB81E58CBD089580912C
:10054000CE008AE00E94470C8091C80087FFD1CF7F
:100550008091C80087FDF3CF8091C80087FFF8CF56
:10056000EECFEF92FF920F931F93CF93DF93EC01A7
:1005700081E0CD32D80750F5C832D105B0F588E218
:1005800090E0909377048093760490938304809313
:1005900082040E94721524E234EF30938604209383
:1005A000850482E080939100809185049091860477
:1005B000909581959F4F9093860480938504DF9159
:1005C000CF911F910F91FF90EF9008958CE291E0F1
:1005D00090937704809376049093830480938204AD
:1005E0000E9472152DE830E2D8CFD0937704C093E3
:1005F0007604D0938304C0938204CE010E947215C6
:100600009E0140E050E060E070E788E399E30E94DB
:100610009041B901CA01969587957795679596950A
:10062000879577956795969587957795679526E051
:1006300030E040E050E00E94904179018A01C80119
:10064000AA27BB279C01887F892B09F45FC0C901B9
:10065000807F892B99F0C901807E892BF1F0C90137
:10066000807C892B49F1C9018070892BA1F1207010
:100670003C7F232BE1F11092910096CFF4E0169588
:100680000795F794E794FA95D1F7F0928604E092F3
:10069000850486E08093910087CFE5E01695079565
:1006A000F794E794EA95D1F7F0928604E0928504F6
:1006B00087E08093910078CF76E016950795F794C0
:1006C000E7947A95D1F7F0928604E092850483E06E
:1006D0008093910069CFBB27A12F902F8F2D9093EE
:1006E00086048093850484E0809391005DCF5AE076
:1006F00016950795F794E7945A95D1F7F0928604EA
:10070000E092850485E0809391004ECFA3E016959A
:100710000795F794E794AA95D1F797013ECF85E026
:1007200090E00E9435020E94B10280918504909170
:100730008604909379048093780410922D04E1E765
:10074000F0E08081816080838091760490917704CD
:1007500090938A0480938904089585E20E949511FC
:10076000E1E7F0E080818E7F80830895AF92BF92B1
:10077000CF92DF92EF92FF920F931F93DF93CF936D
:10078000CDB7DEB760970FB6F894DEBF0FBECDBF12
:100790000E946B020E948F0380916E0082608093A2
:1007A0006E0083E084BD85BD8AEF87BD82E596E05B
:1007B0009093950680939406F999FECF82E090E09D
:1007C00092BD81BDF89A80B5982F937090932C04B8
:1007D0008295817080936404F999FECF87E090E060
:1007E00092BD81BDF89A80B5882311F0813208F05E
:1007F00080E180930002F999FECF83E090E092BD02
:1008000081BDF89A80B58F7080939404F999FECFDA
:1008100084E090E092BD81BDF89A80B58F7080939E
:10082000930488E090E00E94350280938404209134
:10083000760430917704280F391F30937B0420937E
:100840007A0485EB9BE390938C0480938B0483E381
:1008500093E1909392048093910485E694ED9093B4
:100860008804809387040E94E0000E94E0000E94B8
:10087000E000BC0188E090E00E945A02F999FECFA6
:100880008AE090E092BD81BDF89A90B5892F8F7073
:1008900080938D0480918D04833010F010928D042C
:1008A00092959F709F5F9093900480919004823006
:1008B00008F4DDC00E949428789400E010E01DC088
:1008C0008091C1040E942F120E946113C801849676
:1008D00068E270E00E947D410E94FA140E94951126
:1008E00080E10E94470CC80187709070892B69F0E5
:1008F0000F5F1F4F0C32110579F0083208F7802F77
:100900000E94FA140E945D11DBCF0E94B0100F5FAD
:100910001F4F0C32110589F70E940C120E946113BF
:100920000E94B01080E00E94EB0E882331F083E03B
:100930000E94EB0E882309F0E6C083E00E94EB0ED4
:10094000882309F098C08091C1048093AB0610926F
:10095000EC0610927F051092080681E080930E0647
:1009600010920F068091AB066091EC06409108064C
:1009700020910E0602E516E00E941A2860910806F2
:10098000C8010E9428250E94B3240E94B0108091C3
:100990003404836080933404109235048091BC0445
:1009A000873009F461C0883030F5833009F444C0E1
:1009B0008430A8F5882309F445C0813009F43FC08C
:1009C0000E94B0100E94B3248823F9F68091BC04E1
:1009D0008630B1F781E00E94170F882389F380E009
:1009E0000E94EB0E882361F30E940C120E94611397
:1009F000E0E0F0EF19948C30A1F18D3038F48830BC
:100A000039F18B30E9F60E94471EBFCF8E30E9F0F6
:100A10008E3078F08F30A1F60E94AA28B6CF8430AD
:100A200029F0853069F60E949C2DAFCF0E94EB180B
:100A3000ACCF0E942D40A9CF0E94D620A6CF0E9405
:100A4000C839A3CF0E947A0DA0CF0E944D159DCF2B
:100A50000E940C120E94B0100E94B3248823D1F38C
:100A600094CF0E94AD3791CF0E948C228ECF82E02E
:100A7000809390041FCF8CE00E94EB0E882309F432
:100A800062CF7E010894E11CF11CBB2491E1C92EC8
:100A9000D12CCC0EDD1E8FE0A82E87010E94E00035
:100AA000F801908381830E5F1F4F0C151D05B1F770
:100AB000F70104C031960E171F0791F02081822F95
:100AC00090E08F7090700D9724F0822F8F7080834C
:100AD000282F2D3079F78E2F8E198F3009F072C0A4
:100AE00080E060E04B2D21E087010E94CD2785E565
:100AF0000E9419150E946113B394F0E8BF1669F6BD
:100B00000E940C1220CF10922C0410926404609169
:100B1000640470E06170707062957295707F7627E2
:100B2000607F762782E090E00E9450020E94942825
:100B3000109294041092930483E090E060E00E948D
:100B4000500284E090E0609193040E94500288E794
:100B500090E0909377048093760485E090E068E7D6
:100B600070E00E945A0280E18093000260910002CE
:100B700087E090E00E94500210928D0488E08093FC
:100B800090048091900460918D0490E0019782958B
:100B90009295907F9827807F9827682B8AE090E035
:100BA0000E94500210E082E20E94C91183E20E947A
:100BB000C9110E94611382E30E94470C1F5F183223
:100BC00091F79ECFA08276CFCF92DF92EF92FF92E5
:100BD0000F931F93F89480912C04813009F41AC26A
:100BE00080916D04813009F4F8C180912F04863022
:100BF00060F010922F04809130048F5F8093300456
:100C0000809131048F5F8093310480913104882377
:100C100041F08091310490E083709070892B09F449
:100C2000D6C180913204883038F01092320480911D
:100C30002C04882309F4AFC1809131048F70809314
:100C400031049091300480910002981798F010922E
:100C50003004809133048F5F809333049091330488
:100C600080919004981708F093C1809134048260B9
:100C7000809334048091F906882329F4809130040C
:100C8000882309F47BC180913004882329F4809162
:100C90006D04823009F467C280912C048823F1F43A
:100CA00090913D048091E703981710F010923D0455
:100CB00080913D0480FF4DC25C9880913D0480FF8F
:100CC0000DC080913D048F5F80933D0478941F9107
:100CD0000F91FF90EF90DF90CF90089580916E0478
:100CE0002091E7034091E70390E030E0240F311DAD
:100CF0008217930714F010926E0480916E04609135
:100D0000E70366950E945D41992309F496C0DD24AE
:100D10008091BC04873009F49CC0883008F08CC1F5
:100D2000833009F496C0853009F493C0813009F40A
:100D300090C080916D04823009F4CCC28091F90694
:100D4000882321F082E0D81609F4CFC28091F906F9
:100D5000882309F4BBC280915A048F7080935A048F
:100D60008091310490E08370907002970CF4D0C1B0
:100D700085E20E94951180915A0490E083709070F2
:100D800002970CF4C2C18FEF8093520480916304E8
:100D9000882309F08AC180916C04882329F080910E
:100DA0003504882309F0BBC180913604882309F0FB
:100DB0006AC10E946113DD2031F080912D048F5FA4
:100DC000817080932D04209182043091830480915E
:100DD0007604909177042817390719F0C9010E9409
:100DE000B10280916E048F5F80936E048091ED0656
:100DF0008F5F8093ED0680912F048F5F80932F0487
:100E000080913D048F5F80933D042091ED06809199
:100E1000E70330E0869586954CE0849FC00111245D
:100E20002817390714F01092ED0678941F910F914E
:100E3000FF90EF90DF90CF90089580912D0488234C
:100E400009F46AC1DD24D3948091BC04873009F091
:100E500064CF81E0D81609F494C182E0D81609F075
:100E600068CF80915A048F5F80935A048091F9066D
:100E7000882309F47DC080918005882309F51092AC
:100E8000ED0680918405882349F48091EF0688233C
:100E900029F080916304882309F09AC380910806A1
:100EA00060915006680F80919406909195060E947B
:100EB000282510925A0480915E04882309F4D1C237
:100EC00080918005E0919406F0919506E80FF11D60
:100ED0008081809375048091810480938004809147
:100EE000750480748093810480916304882309F0E1
:100EF0005DC2809175048F708F3009F4AAC2809111
:100F000075048F708F3071F0809175040E944C25AC
:100F100090919A0660918004409175044078890F01
:100F20000E94CC188091BC04833009F432C28091B5
:100F3000BC048730E9F480913604813009F440C361
:100F40008091680590916905E0917905F0E0EE0FD8
:100F5000FF1FEF5FFD4F6081718182959295907FB9
:100F60009827807F98270E946941862F0E943A1215
:100F700080913404816080933404DBCE80916D04D1
:100F8000823009F080CE10926D040E94B12B7BCE8E
:100F9000109233046ACE20917604309177048091C8
:100FA000890490918A042817390709F445CE85E20F
:100FB0000E945D11609176047091770470938A04A9
:100FC0006093890485E090E00E945A0235CE8091BA
:100FD00032048F5F8093320424CE8091F9068823F7
:100FE00009F0BCC00E94B12B80912C04882309F029
:100FF000B7C0109232048091320480933104809102
:101000003104809330048091300480932F04109237
:101010003304A6C080916C04882309F4E1CD0E94BA
:101020007C0E882309F09EC10E948E0E882309F44D
:10103000D7CD0E944E2BD4CD883029F08B508330F1
:1010400008F077CE06CF81E0D81609F47DC182E0A2
:10105000D81609F06ECE8091740480932E0480918E
:101060007304809374040E94AF0080937304809192
:1010700074048F7360E040E00E94CC188091740487
:101080000E94730C56CE0E940B158091310480FD96
:1010900090CEE0913104E695F0E0E370F070E45812
:1010A000FB4F80810E94001584CE8CE20E944C256B
:1010B000982F80915A048111945F8091ED068823C6
:1010C00041F480916404882309F446C183E20E94BC
:1010D0005D118091ED06823009F05DCE809164044F
:1010E000882379F480916104823008F44EC18091A4
:1010F0000C060E944C2540910C06407860E00E944E
:10110000CC1883E20E94951146CE109252043ECE36
:1011100085E20E945D112FCEB2E0DB2EF9CD8091E9
:101120008D04813009F4E5C080918D04882309F095
:101130003BCE8091340480FF37CE809134048E7F83
:10114000809334040E942112809180050E942F1206
:101150002BCE5C9A88EF0E94DA0CAFCD0E944E2B0A
:1011600010926D0442CD8091BC04853009F494CD79
:1011700010926E0410922D041092800510926D044E
:101180008BCD809184058F5F809384058091F906D3
:10119000882309F4CECD809180058F5F80938005F0
:1011A000909180058091E903981710F010928005C6
:1011B00080918005882309F06EC08091BC04833043
:1011C00009F4A7C010E08091BC04873009F405C180
:1011D00081E00E94F724809150068F5F8093500633
:1011E000C09050069091500680910E06981708F412
:1011F00043C080915E04882319F481E080936B04DE
:101200008091BC04813009F4D1C18091BC048C3040
:1012100009F470C182E00E94F72410928405809145
:101220006304882369F0809161048093EF068091C4
:10123000EF06882329F01092610481E080937E05F7
:10124000109250068091BC04833009F457C18091FC
:10125000BC04873009F428C180910F06882309F067
:101260000FC19091EC0680917F05981729F080912D
:101270005E04823008F4E0C18091500690E08295CF
:101280009295907F9827807F98278E5A994F9093B8
:1012900095068093940680916304882309F049CDD4
:1012A00080918005E0919406F0919506E80FF11D7C
:1012B000808180937504809175048F708F3009F45C
:1012C00084C0809181040E94E31833CD81E20E94A2
:1012D000951141CD81E20E94951180912F0463E028
:1012E0000E945D41992309F036CD81E20E945D1193
:1012F00032CD8091340481FF17CF809134048D7FEB
:10130000809334040E942112809133040E942F1292
:101310000BCF8091680590916905019690936905BE
:101320008093680520916805309169058091730567
:10133000909174052817390708F444CF1092690575
:101340001092680511E03FCF80E00E94E318809181
:1013500074040E94B20CEDCC892F60E040E00E9442
:10136000CC18B4CE0E94B12B10923204809132047A
:101370008093310480913104809330048091300453
:1013800080932F04109233044FCE80E00E94E31824
:10139000B8CE80913604813009F0C9CD80916805BE
:1013A0009091690501960E94EB01C1CD80910806DC
:1013B00060910E064091810520910F0600918505F0
:1013C000E0907F050E945314ADCD80918104882365
:1013D00009F0EFC01092810474CF809159048130DC
:1013E00009F0F6CE6091EC06809108064091500617
:1013F00020919A06480F80E795E00E944B1A809151
:1014000079056091680570916905409170050E94A9
:10141000B11A8091680590916905019690936905CC
:1014200080936805E0917905209168053091690500
:10143000F0E0EE0FFF1FEF5FFD4F808191812817D5
:10144000390708F4C5CE1092590483E20E94951121
:10145000BFCE809175048F708093750410928104C3
:101460004ECD8091080660910E0640918105209135
:101470000F0600918505E0907F050E94531420CD52
:101480000E94E42480915E04823008F0F5CE8091C1
:10149000AB066091EC064091080620910E0602E52D
:1014A00016E00E941A28E8CE80915904813009F094
:1014B000D3CE80916C05882309F0C3C080916D055F
:1014C000882309F4C9CE10926D0580917905609149
:1014D0006805709169056C190E94781A80917905E8
:1014E0000E940B1B90937B0580937A0580E00E94FD
:1014F0009511B2CE81E080936B048CCE80916C0507
:10150000882309F080C080916D05882309F455C0B7
:1015100010926905109268058091B704809379054F
:10152000809179050E94141B909374058093730534
:10153000809179050E940B1B90937B0580937A051F
:1015400020917A0530917B05809173059091740507
:101550002817390720F010927B0510927A058091A8
:101560006D05882309F05AC080917905609168055E
:10157000709169050E94651B8093700580917905C3
:101580006091700547EC55E02FE735E001E815E084
:1015900073E9E72E76E0F72E0E942B1A81E0809304
:1015A0000F068091930680939A0651CE80936B0428
:1015B0002CCE81E00E94E3180DCF112381F2A8CF39
:1015C000809168059091690501960E94EB01B8CC65
:1015D00081E00E94E31880E00E94E31860910E060B
:1015E00082E596E04CEA56E026E835E00E94572670
:1015F000109263048AE00E9468251092810482E0C0
:101600000E94470C4BCC10926C0510926905109209
:10161000680583E20E94951111E075CF10926D0567
:1016200080917A0590917B05909369058093680578
:1016300080E00E94951198CF80917F058093EC0601
:1016400026CF1092590410926C0580917905609113
:101650006805709169050E94881A809179050E9439
:10166000141B909374058093730583E20E94951177
:1016700025CF1F920F920FB60F920BB60F92112427
:101680001F932F933F934F935F936F937F938F930A
:101690009F93AF93BF93EF93FF9320B1227090B1CC
:1016A00080918F042817F1F0892F8170222309F48B
:1016B0007AC0882309F47AC08091820490918304CF
:1016C0000197909383048093820431E08D329307D5
:1016D00008F47AC08CE291E09093830480938204B2
:1016E00020938F04809146048F3F29F08091460417
:1016F0008F5F80934604809147048F3F29F080914B
:1017000047048F5F80934704809171049091720425
:101710008F5F9F4F49F08091710490917204019600
:1017200090937204809371048091550490915604B3
:101730008F5F9F4F49F08091550490915604019618
:10174000909356048093550410912C04113009F4A1
:1017500045C08091400490914104892B81F0809193
:101760004004909141040197909341048093400478
:101770008091400490914104892B09F45C98FF9179
:10178000EF91BF91AF919F918F917F916F915F91F9
:101790004F913F912F911F910F900BBE0F900FBE55
:1017A0000F901F901895882309F486CF80918204AA
:1017B000909183040196909383048093820431E096
:1017C0008D32930708F086CF889708F089CF88E29A
:1017D00090E0909383048093820482CF99B1929594
:1017E000917080914404882319F090934404C7CFEA
:1017F0009923D9F380913E0490913F0401969093F0
:101800003F0480933E0410923F0410923E040E94D5
:10181000E40588EF0E94DA0C10934404B0CF1F92C5
:101820000F920FB60F920BB60F9211242F933F9386
:101830004F935F936F937F938F939F93AF93BF93D8
:10184000EF93FF93809178049091790490939500A1
:1018500080939400809185049091860490937904FC
:10186000809378040E94E405FF91EF91BF91AF91BE
:101870009F918F917F916F915F914F913F912F91A8
:101880000F900BBE0F900FBE0F901F90189520EA7F
:101890003FE0E22FF32F3197F1F78A95D1F70895C2
:1018A000882309F41EC09AEF20EA3FE0E22FF32FCD
:1018B0003197F1F79A95D1F7E22FF32F3197F1F79E
:1018C0009A95D1F7E22FF32F3197F1F79A95D1F747
:1018D000E22FF32F3197F1F79A95D1F7815009F064
:1018E000E5CF08950895282F909193048091C0002A
:1018F00085FFFCCF90699093C600822F90E08F7394
:101900009070892BB1F48091C00085FFFCCF1092BC
:10191000C600822F829586958695837080FD19C0BA
:10192000909123028091C00085FFFCCF9093C60068
:1019300008958091C00085FFFCCF822F8F73875E52
:101940008093C600822F829586958695837080FF4E
:10195000E7CF909121028091C00085FFFCCF90934A
:10196000C6000895282F909193048091C00085FFB0
:10197000FCCF90689093C600822F90E08F73907098
:10198000892B39F48091C00085FFFCCF1092C600EE
:1019900008C08091C00085FFFCCF2F73275E209385
:1019A000C600909122028091C00085FFFCCF9093E9
:1019B000C6000895982F8091C00085FFFCCF9093BA
:1019C000C60080E090E0089590913B0480913C0433
:1019D00020E030E0981711F021E030E0C9010895CF
:1019E00090913B0480913C049817D1F3F894909126
:1019F0003B04E92FF0E0EB56FB4F80819F5F909313
:101A00003B0490913B049F7190933B04789490E049
:101A1000089590913B0480913C04981729F00E940E
:101A2000F00C482F87FD03C040E0842F0895582F05
:101A300052955F705F30C9F3282F30E02F703070FF
:101A40008091940490E02817390771F75093380477
:101A5000ECCF909193048091C00085FFFCCF906BF8
:101A60009093C6008091C00085FFFCCF8BE78093E8
:101A7000C6008091C00085FFFCCF1092C60008957B
:101A800080912C04823049F08091C00085FFFCCF0A
:101A90008CEF8093C6000E94290D089590912E042A
:101AA0008913089580E00E94E3188FEF80932E043D
:101AB00008951F93182F962F6623B9F060E0809148
:101AC0002E048F3F09F061E0953648F4812F89514B
:101AD00040E00E94CC1810932E041F910895812F8E
:101AE000895141E00E94CC18F6CF60E00E944E0D73
:101AF0001F9108951F930E942112809194040E94C7
:101B00002F120E94B01084E60E94470C0E94B01071
:101B100084E60E94470C0E94B0108FEF80932E0441
:101B20000E94B0100E94B324882301F590913B04D9
:101B300080913C049817A1F30E94F00C482F87FD78
:101B400019C080913804883039F1893049F747FD50
:101B500030C0142F0E94F00C682F812F0E94590D65
:101B60000E94B0100E94B324882301F30E94290D23
:101B70001F910895582F52955F705F30B9F0282F4C
:101B800030E02F7030708091940490E0281739076E
:101B900069F010923804C4CF47FD0FC0142F0E9483
:101BA000F00C682F812F0E944E0DBACF509338044D
:101BB000C8CF0E94F00C182FCDCF0E94F00C182F28
:101BC000EECF1F920F920FB60F920BB60F92112409
:101BD0002F933F934F935F936F937F938F939F9335
:101BE000AF93BF93EF93FF939091C6009A3F09F490
:101BF00042C09C3FA9F1983F09F44AC080913C043F
:101C0000E82FF0E0EB56FB4F90838F5F80933C040E
:101C100080913C048F7180933C0490913C048091AE
:101C20003B04981751F480913B048F5F80933B04F1
:101C300080913B048F7180933B04FF91EF91BF91A2
:101C4000AF919F918F917F916F915F914F913F9154
:101C50002F910F900BBE0F900FBE0F901F901895F5
:101C600080916C04882349F380912C04823029F7F9
:101C70000E944E2BE2CF80916C048823F1F2809178
:101C80002C048230D1F60E94B12B0E948900D5CF5E
:101C9000809171049091720490932B0480932A0494
:101CA000109272041092710480912C04823029F6F3
:101CB0008091390490913A04019690933A0480936C
:101CC00039045C9A8091C00085FFFCCF88EF809337
:101CD000C6000E94E40580912A0490912B049695F9
:101CE000879580934004A9CF5F9A089580912C0432
:101CF000813009F05F98089599B1991F9927991F2C
:101D000080914204882311F4992321F49093420492
:101D100080E008959093420481E0089599B1991F5D
:101D20009927991F80914304882311F0992321F06A
:101D30009093430480E008951092430481E0089555
:101D40008AB1806F8AB98BB18F708BB908958AB1CF
:101D50008F708AB98BB18F708BB90895AC01F894EC
:101D600028980000000000000000289A20E030E0E1
:101D70001EBC0DB407FEFDCF8EB5FA01E20FF31FB6
:101D800080832F5F3F4F2330310591F7789408957A
:101D900016980895169A089520B1269526952F70C5
:101DA000822F90E02695322F369536952270322B71
:101DB000880F991F282F2470322B880F991F880FA6
:101DC000991F8870382B8FE0831B089580B186950A
:101DD00086958F700895282F883188F4E82FE6952E
:101DE000E695E695F0E0EE53FB4F808190E027709A
:101DF00002C0959587952A95E2F78170089580E055
:101E00000895282F883188F4E82FE695E695E69521
:101E1000F0E0E754FB4F808190E0277002C0959579
:101E200087952A95E2F78170089580E00895282F1C
:101E3000883188F4E82FE695E695E695F0E0E354DE
:101E4000FB4F808190E0277002C0959587952A9579
:101E5000E2F78170089580E008958091C20488239C
:101E600021F48091C304882319F090E0892F08950C
:101E700090E08091C4048823C9F791E0892F0895E8
:101E8000282F8831A0F4482F46954695469527700F
:101E900081E090E0382F01C0330F2A95EAF7A42F94
:101EA000B0E0FD01E754FB4F8081832319F420E06B
:101EB000822F0895232F30E020953095AE53BB4FED
:101EC0008C9190E028233923232B89F7342F3F5F0F
:101ED000832F63E00E945D41E92FF0E0EE53FB4F5A
:101EE0008081882321F720E0832F8F5F0E945D414E
:101EF000E92FF0E0EE53FB4F80818823C9F621E003
:101F0000D7CF1F93CF93DF93C6E3D2E010E0888151
:101F10000E94EB0E882329F41F5F21961D30B9F72C
:101F20001FEF812FDF91CF911F9108951F93CF93C2
:101F3000DF93C6E3D2E010E088810E94010F88237E
:101F400049F41F5F21961D30B9F780E0DF91CF91F2
:101F50001F910895812F8F5FDF91CF911F91089579
:101F60001F93CF93DF93C6E3D2E010E088810E94F5
:101F7000170F882349F41F5F21961D30B9F780E0C1
:101F8000DF91CF911F910895812F8F5FDF91CF91C6
:101F90001F9108951F93CF93DF93CEE2D2E010E01C
:101FA00088810E94EB0E882349F41F5F2196183028
:101FB000B9F780E0DF91CF911F910895812F8F5F56
:101FC000DF91CF911F9108951F93CF93DF93CEE2BE
:101FD000D2E010E088810E94010F882349F41F5F3E
:101FE00021961830B9F780E0DF91CF911F910895C5
:101FF000812F8F5FDF91CF911F9108951F93CF9312
:10200000DF93CEE2D2E010E088810E94170F882390
:1020100049F41F5F21961830B9F780E0DF91CF9126
:102020001F910895812F8F5FDF91CF911F910895A8
:10203000CF93DF93CEE2D2E088810E94EB0E88231B
:1020400049F4219682E0C633D807B1F780E0DF91EA
:10205000CF91089581E0DF91CF910895FF920F9382
:102060001F93CF93DF93CEE2D2E0FF2400E006C0BF
:102070000F5F219682E0C633D80789F01881812F3F
:102080000E94EB0E8823A1F7812F0E94170F88234F
:1020900081F3F394219682E0C633D80779F781E083
:1020A000F81639F080E0DF91CF911F910F91FF90EA
:1020B000089580E00730B9F781E0F5CF1F93CF9303
:1020C000DF93C4E2D2E010E088810E94010F8823F0
:1020D00049F41F5F21961A30B9F780E0DF91CF9164
:1020E0001F910895812F8F5FDF91CF911F910895E8
:1020F0008091450410924504089580E00895382F9A
:10210000883100F5282F277081E090E0982F01C0DA
:10211000990F2A95EAF7832F869586958695A82F9D
:10212000B0E0FD01E754FB4F8081892369F4FD0194
:10213000E354FB4F8081892371F4AE53BB4F8C91E4
:10214000982339F480E00895832F0E94331482E0AD
:10215000089583E00895832F0E943B1481E0089541
:10216000EF92FF920F931F93DF93CF9300D000D095
:10217000CDB7DEB71092B9041092BD041092BA0424
:102180001092BE041092BB041092BF0480914604CA
:102190008A3068F426960FB6F894DEBF0FBECDBF26
:1021A000CF91DF911F910F91FF90EF9008951092C2
:1021B000460416987E010894E11CF11CC7010E9498
:1021C000AE0E8091C2048C838091C3048D83809174
:1021D000C4048E8360E070E001E010E0E62FE69535
:1021E000E695E695F0E0CB0187709070980102C00B
:1021F000220F331F8A95E2F7C901AF014E535B4F9F
:10220000D701AE0FBF1F3C91EB53FB4F2081232B17
:1022100028238095FA0130818323282B20836F5F48
:102220007F4F68317105D1F60E94CC0E982F96959C
:102230009093C1048093B704169A40E050E0BE0129
:102240006C5F7F4FDA01AB53BB4FF701E40FF51F13
:1022500080818C93FB01E40FF51F2081FA01EE537E
:10226000FB4F9081FA01E754FB4F822F8095892321
:102270008083FA01E354FB4F9095922390834F5F44
:102280005F4F43305105F1F690B1969596959F704A
:102290008091B504891721F0109247049093B504FA
:1022A000809147048F3630F09093B6048091B60445
:1022B0008093B5040E9461136DCF282F8832C0F43B
:1022C000E82FE695E695E695F0E0277081E090E04E
:1022D00001C0880F2A95EAF7DF01A85BBB4F2C915C
:1022E000282B2C93E35BFB4F8095208182238083F6
:1022F0000895282F8832C0F4E82FE695E695E695F4
:10230000F0E0277081E090E001C0880F2A95EAF79D
:10231000DF01A35BBB4F2C91282B2C93E85BFB4F79
:1023200080952081822380830895282F8832C8F4E5
:10233000E82FE695E695E695F0E0277081E090E0DD
:1023400002C0880F991F2A95E2F78095DF01A85BEC
:10235000BB4F2C9128232C93E35BFB4F20818223DE
:1023600080830895282F883298F4E82FE695E69523
:10237000E695F0E0E35BFB4F277081E090E002C060
:10238000880F991F2A95E2F7809520818223808308
:102390000895282F883290F4E82FE695E695E69583
:1023A000F0E0E85BFB4F277081E090E002C0880F0F
:1023B000991F2A95E2F72081282720830895E82F86
:1023C000883298F4282F277081E090E002C0880FAF
:1023D000991F2A95E2F7E695E695E695F0E0E35B2E
:1023E000FB4F20812823822F089520E0822F08951B
:1023F000982F969596959695E8E4F4E0E90FF11DEF
:10240000208130E0877002C0359527958A95E2F7E4
:1024100021703070C901089510924C0410924B0441
:1024200010924A04109249041092480410925104E8
:102430001092500410924F0410924E0410924D04CA
:102440000895CF93DF93C2EAD2E089910E9495115B
:1024500082E0C23BD807C9F7DF91CF910895803160
:1024600008F00895E82FF0E0EE55FD4F80810E94BE
:102470005D1108950F931F93CF93DF93082FC2EA46
:10248000D2E010E007C088810E945D111F5F219695
:10249000103149F01017B8F388810E9495111F5F21
:1024A00021961031B9F7DF91CF911F910F910895C7
:1024B000803108F00895E82FF0E0EE55FD4F80815F
:1024C0000E9479110895803110F080E00895E82F7E
:1024D000F0E0EE55FD4F80810E94F81108958031A3
:1024E00010F080E00895E82FF0E0EE55FD4F808178
:1024F0000E94DF110895883108F00895E82FF0E078
:10250000E358FD4F80810E945D110895883108F0E5
:102510000895E82FF0E0E358FD4F80810E94791183
:102520000895883108F00895E82FF0E0E358FD4F52
:1025300080810E9495110895CF93DF93CDE7D2E07B
:1025400089910E94951182E0C539D807C9F7DF91BA
:10255000CF910895E82F8150883008F00895F0E079
:10256000EC58FD4F80810E945D1108950F931F93D9
:10257000CF93DF93082FC5E7D2E011E007C0888131
:102580000E9495111F5F2196193069F01017B9F755
:10259000E12FF0E0EC58FD4F80810E945D111F5F3C
:1025A0002196193099F7DF91CF911F910F910895DE
:1025B000E82F8150883008F00895F0E0EC58FD4F86
:1025C00080810E9495110895E82F8150883008F08D
:1025D0000895F0E0EC58FD4F80810E947911089534
:1025E000E82F8150883010F080E00895F0E0EC583A
:1025F000FD4F80810E94DF110895E82F81508830BF
:1026000010F080E00895F0E0EC58FD4F80810E94CA
:10261000F8110895CF93DF93C5E7D2E089910E9426
:10262000951182E0CD37D807C9F7DF91CF91089592
:102630008D3008F00895E82FF0E0EB56FD4F8081D3
:102640000E945D1108958D3008F00895E82FF0E0A4
:10265000EB56FD4F80810E94951108958D3008F052
:102660000895E82FF0E0EB56FD4F80810E9479112C
:102670000895E5E9F2E0E80FF11D80810E94DF1185
:102680000895CF93DF93C5E9D2E089910E94951117
:1026900082E0C23AD807C9F7DF91CF9108950E942E
:1026A000411384E00E94951183E00E94951188E017
:1026B0000E94951181E00E94951182E00E9495117F
:1026C0000895F894179820E030E090915204F901B1
:1026D000E35BFB4F80819823F901E85BFB4F80812E
:1026E000982B9EBD0DB407FEFDCF2F5F3F4F2530C9
:1026F000310559F7179A78940895E8E4F4E0ADE4C9
:10270000B4E080819D91892B819384E0ED34F807BA
:10271000C1F70895E8E4F4E0ADE4B4E09D9190954C
:1027200080818923819384E0ED34F807B9F7089517
:10273000E8E4F4E0ADE4B4E020819C91892F8223A9
:1027400019F09095922390831D92319684E0ED3498
:10275000F80791F708951F93182F84E00E949511B0
:10276000123061F083E00E94951183E00E94B21163
:10277000113071F01F3F39F01F91089583E00E94DE
:1027800079111F91089584E00E945D111F910895B1
:1027900083E00E945D111F9108950F931F93CF93C3
:1027A000DF93182F87FD50C086E10E949112812F80
:1027B000829586958695837080FF29C085E10E9469
:1027C0007B121F7349F11731A0F58FEF0E94AB13F5
:1027D00084E10E949112012F10E0CBE0D0E0C017FD
:1027E000D10731F0FE01E657FD4F80810E9495111F
:1027F0002196C831D10599F706571D4FF801808100
:102800000E945D11DF91CF911F910F91089585E195
:102810000E9491121F73B9F680E00E94AB130E94D0
:10282000411384E10E947B12DF91CF911F910F91A0
:102830000895143268F0103370F4185181E00E944A
:10284000AB13112329F6EBCF86E10E947B12AFCFA9
:102850001C5080E0F4CF1C3318F4145282E0EFCF08
:10286000105383E0ECCFEDE7F2E0E80FF11D80813B
:102870000E945D110895EDE7F2E0E80FF11D8081FF
:102880000E9495110895E5E7F2E0E80FF11D8081BF
:102890000E945D110895E5E7F2E0E80FF11D8081E7
:1028A0000E9495110895DF92EF92FF920F931F936C
:1028B000CF93DF93F02EDE2C222371F1022F040F31
:1028C000E42EC5E7D2E010E00BC0101758F41F1536
:1028D000D9F088810E945D111F5F2196183049F060
:1028E0001E1598F788810E9495111F5F2196183058
:1028F000B9F781E08D15A0F4DF91CF911F910F9171
:10290000FF90EF90DF900895E12FF0E0EB58FD4F3E
:1029100080810E947911E0CF062F080FE82ED1CFD9
:10292000DD2071F088E00E94951181E00E945D1128
:10293000DF91CF911F910F91FF90EF90DF9008955D
:1029400088E00E945D1181E00E949511DF91CF9196
:102950001F910F91FF90EF90DF900895FF920F93DA
:102960001F93082FF62E84E00E94951183E00E94A9
:10297000951188E00E94951181E00E949511102F19
:1029800004FD34C015FD29C007FD2CC016FD21C073
:102990000E944113FF2099F0802F8F708D3098F0A6
:1029A0008BE10E945D118CE10E945D118FE00E941D
:1029B0005D118EE00E945D118DE00E945D111F91FE
:1029C0000F91FF9008950E9418131F910F91FF908F
:1029D000089581E00E945D11DBCF83E00E945D11CC
:1029E00007FFD4CF88E00E945D11D0CF84E00E9421
:1029F0005D11C8CFE3E4F2E0E80FF11D8081089596
:102A00008A3008F00895E82FF0E0E559FD4F808105
:102A10000E945D110895CF93DF93CBE6D2E08991B8
:102A20000E94951182E0C537D807C9F7DF91CF9191
:102A300008959091480498279093480490914904F0
:102A400098279093490490914A04982790934A04B8
:102A500090914B04982790934B0490914C049827A5
:102A600090934C040895AC0161157105A1F020E02C
:102A7000E0E0A0E0B0E0A40FB51F8C91E827F0E003
:102A8000E654FD4FE0812F5FA22FB0E0A617B707F5
:102A900090F38E2F0895E0E0FCCF0E94B0100E94CA
:102AA000B3248823D1F30895EF92FF920F931F93DD
:102AB000CF93DF937C018B016115710561F0C0E05C
:102AC000D0E0F701EC0FFD1F80810E94CE0121961E
:102AD000C017D107B0F3DF91CF911F910F91FF90F5
:102AE000EF90089522E42093C8041092C90422E0D4
:102AF0002093CA049093CB048093CC04A8ECB4E058
:102B0000E0E08D91E827F0E0E654FD4FE08184E0BD
:102B1000AD3CB807B1F7EC93CD01059766E070E0E6
:102B20000E945415089590E89093C8041092C90427
:102B300021E02093CA048093CB04AAEBB2E09091E9
:102B40003A03FD01E90FF11D90819227FD01E90F84
:102B5000F11D90819827A90FB11D8C918093CC0411
:102B600088EC94E065E070E00E94541508951F928F
:102B70000F920FB60F920BB60F921124DF92EF92C5
:102B8000FF920F931F932F933F934F935F936F93F6
:102B90007F938F939F93AF93BF93CF93DF93EF93E5
:102BA000FF931091CE008091B902882309F46EC082
:102BB0008091550490915604895E934008F080C03E
:102BC00080915304803408F089C0282F2F5FE82FAC
:102BD000F0E0E85FFA4F10832093530410925604FC
:102BE00010925504233008F451C07091080590915B
:102BF000090580E060910A05462F50E0482B592BCB
:102C000030E0CA0104962817390708F43FC09A013A
:102C10002D5F3F4FF901E85FFA4F10812115310513
:102C200009F401C190E0E0E0A0E0B0E0A85FBA4F95
:102C30008C91E827F0E0E654FD4FE0819F5FA92FDB
:102C4000B0E0A217B30790F31E1709F450C0211586
:102C5000310509F4EAC090E0E0E0A0E0B0E0A85F50
:102C6000BA4F8C91E827F0E0E654FD4FE0819F5F7A
:102C7000A92FB0E0A217B30790F38E2F90E00E9427
:102C8000AA011092530480E00E949315FF91EF91E6
:102C9000DF91CF91BF91AF919F918F917F916F9174
:102CA0005F914F913F912F911F910F91FF90EF9066
:102CB000DF900F900BBE0F900FBE0F901F901895D6
:102CC0000E9421120E9461131093080581E08093F5
:102CD00053041092560410925504D8CF0E949315B5
:102CE000109253041092560410925504CFCF7138AD
:102CF00009F492C17238B0F5713109F42BC1723107
:102D000008F096C0713051F1703131F080E00E94CE
:102D1000931510925304BACF6231C1F780910B051D
:102D2000082F10E0000F111F000F111F000F111FBF
:102D300080910C05080F111D02951295107F102728
:102D4000007F1027CDE0D5E08991B8010E94AC1931
:102D50000F5F1F4F85E0CD31D807B1F781E00E94AA
:102D60009315D7CF763809F435C1773808F073C09A
:102D7000723809F484C1753849F64330510509F0B9
:102D8000A5C030910B05932F80E020910C05E22E19
:102D9000FF24E82AF92AD0900D05EAE3ED1508F49E
:102DA000B6CF7093C8041092C904F2E0DF0ED0923F
:102DB000CA048EEFD80E3093CB042093CC04DD20D0
:102DC00071F00DEC14E0E701CE010E94F019F8015A
:102DD00081938F0121969E012E192D15A8F38091C4
:102DE000CA04682F6D5F09F4D5C1A8ECB4E090E087
:102DF0008E5F282F30E027533B4F8D919827E92F86
:102E0000F0E0E654FD4F9081A217B307B1F7E62F2B
:102E1000F0E0E853FB4F90836F5F88EC94E070E044
:102E20000E94541576CFE0E00FCF80E090E027CFEE
:102E3000703409F453C1713409F068CF623009F07D
:102E400065CF90910B0580E020910C05820F911DBC
:102E50000E94B1025ECF7738E9F1783809F056CF99
:102E60007093C8041092C90480910B05813009F455
:102E70006AC1813008F05BC180E18093CB0410927D
:102E8000CC048093CD041092CE0484E047E0A7E008
:102E9000B0E068E070E08093CA0490E020E030E0A9
:102EA000F901E853FB4F80819827E92FF0E0E654C1
:102EB000FD4F90812F5F3F4F241790F3A853BB4FD6
:102EC0009C9388EC94E00E94541523CF80E00E94EC
:102ED00093151FCF80910B05882309F006C142305E
:102EE000510509F014CFE0910C05E43008F00ECF45
:102EF00089E18093C8041092C90480E18093CA04D8
:102F00002E2F30E022953295307F3227207F3227D6
:102F1000ABECB4E0F901EE5AF94F80818D932F5F4D
:102F20003F4F84E0AB3DB807A9F75397E0E08D91A0
:102F3000E827F0E0E654FD4FE081F4E0AB3DBF0749
:102F4000B1F7E093DB04CD01439764E170E00E94A8
:102F50005415DFCE623009F0D9CE80910B05082FD1
:102F600010E0000F111F000F111F000F111F8091A3
:102F70000C05080F111D02951295107F1027007F78
:102F8000102789E18093C8041092C90480E18093DE
:102F9000CA04CBECD4E0C8010E94F01989930F5FFA
:102FA0001F4F34E0CB3DD307B1F7DE015397E0E08C
:102FB0008D91E827F0E0E654FD4FE081CA17DB076A
:102FC000B9F7E093DB0488EC94E064E170E00E94E0
:102FD00054159FCE90910B0580E020910C05E22EB8
:102FE000FF24E82AF92A2EEFD22ED60E63506A3338
:102FF00008F06CCFDD2009F4B1CE0DE015E0E7015B
:10300000F80181918F01BE010E94AC1921969E01A9
:103010002E192D15A8F3A2CE87E190E09093CC0451
:103020008093CB0489EC90E09093CE048093CD0400
:10303000E2EBF2E0AFECB4E081918D9322E0E83B6B
:10304000F207D1F781E88093C8041092C9048AE09E
:103050008093CA04A8ECB4E0E0E08D91E827F0E0AA
:10306000E654FD4FE08134E0A53DB307B1F7EC93A2
:10307000CD010D976EE070E00E9454154ACE4230AB
:10308000510509F023CF30910B05332309F468C0B3
:1030900090910C0520E082E88093C8041092C90446
:1030A00083E08093CA043093CB049093CC042093A4
:1030B000CD04A8ECB4E0E0E08D91E827F0E0E65420
:1030C000FD4FE08184E0AE3CB807B1F7EC93CD0151
:1030D000069767E070E00E9454151BCE809176043D
:1030E000909177040E94721514CE813009F00ECEB3
:1030F0004231510509F00ACEE0910C05E43008F0A8
:1031000005CE2E2F30E0ADE0B5E022953295307F30
:103110003227207F32278D91F901EE5AF94F8083B3
:103120002F5F3F4F85E0AD31B807A9F717CE883044
:1031300009F0ECCD81E08093CB0444E0A4E0B0E062
:1031400065E070E0A8CE88E08093CB0480E18093B6
:10315000CC0482E045E0A5E0B0E066E070E09BCE04
:1031600090910C05973860F4953870F4993181F09E
:10317000993120F0892F8158823030F020E08BCFB8
:10318000973821F09838D1F721E085CF24E083CF1C
:1031900020E181CF90E03BCE2C98803408F08FE383
:1031A000611160E4442349F090E0882349F0682BE2
:1031B000962B98B92C9A2D9A089590E88823B9F700
:1031C000962B98B90895882319F42D982C98089572
:1031D000469A2C9808959F92AF92BF92CF92DF9219
:1031E000EF92FF920F931F93CF93DF930E942112D0
:1031F000809193040E942F120E94B0100E947810B8
:10320000CC24DD249924AA240E94B0100E94B32467
:10321000882309F07CC08C2D0E94AB13C601880F57
:10322000991F8C0D9D1DE82EEE0CEE0CB92CB2945E
:10323000BB0CBB0C80ECB82287E1E80EC0E0D0E00C
:1032400009C0802F0E94170F882319F52196CD30D1
:10325000D10559F1FC2EFE01E654FC4F0081802F70
:103260000E94010F882369F31E2D1C0F812F6A2DE8
:10327000492D0E94CC188B2D812B0E94730C8C2F12
:103280000E941813AA24A394802F0E94170F88234A
:10329000E9F28E2D8F0D8B290E94B20C8F2D0E948A
:1032A00023132196CD30D105A9F68FE00E94010F9E
:1032B0008823D9F182E0C816D1040CF449C085E115
:1032C0000E94010F882351F080E0992009F481E0E9
:1032D000982E8823C9F181E00E945D1186B190E0AB
:1032E0008F739070892B09F48FCF0E942D0F882344
:1032F00009F48ACF80E00E94E3180E944113AA24B7
:103300000E94B0100E94B324882309F484CF0E9445
:10331000290DDF91CF911F910F91FF90EF90DF90DA
:10332000CF90BF90AF909F9008958EE00E94010FC4
:10333000882329F28FEFC8168FEFD80609F4BFCF84
:103340000894C108D108BBCF81E00E949511C6CF77
:103350000894C11CD11CB3CF282FF89495E028986D
:1033600000000000000000009EBD0DB407FEFDCF70
:1033700000000000000000001EBC0DB407FEFDCFE1
:103380008EB5289A000000000000000080FDE7CF05
:1033900028980000000086E08EBD0DB407FEFDCF2A
:1033A00000000000289A000000000000000028989B
:1033B0000000000082E08EBD0DB407FEFDCF7EBD93
:1033C0000DB407FEFDCF6EBD0DB407FEFDCF2EBDC3
:1033D0000DB407FEFDCF00000000289A78940895F0
:1033E000382FF89425E02898000000000000000025
:1033F0002EBD0DB407FEFDCF000000000000000050
:103400001EBC0DB407FEFDCF8EB5289A000000004B
:103410000000000080FDE7CF28980000000083E056
:103420008EBD0DB407FEFDCF9EBD0DB407FEFDCFD2
:103430003EBD0DB407FEFDCF000000001EBC0DB464
:1034400007FEFDCF8EB5289A78940895892F8F7145
:1034500084FD806E0895EF92FF920F931F93FA01FF
:10346000D90186958083862F90E08F709070959516
:10347000879595958795959587958C93862F8770D9
:10348000F801808362956F70F70160831F910F913F
:10349000FF90EF900895FC0130E022953295307F47
:1034A0003227207F322720838081660F660F660FC8
:1034B000640F6F70862B8083089580915704882352
:1034C00049F087FD0EC083E00E945D1184E00E94F8
:1034D0009511089583E00E94951184E00E94951152
:1034E000089583E00E94951184E00E945D11089583
:1034F000962F803110F08FEF0895682F70E0660FDF
:10350000771F6F5F734F892F0E94AC1980E0089579
:103510009B01803120F5682F70E0FB01EE0FFF1F4B
:10352000E953FC4F8081918128173907A0F000975B
:1035300049F08150660F771F6050744F0E94AC199C
:1035400080E0089580E0660F771F6050744F0E94FE
:10355000AC1980E00895C901009759F7F3CF8FEFB8
:103560000895803198F470E06050784F90E0002426
:10357000969587950794969587950794982F802D13
:10358000680F791F8CE06030780710F08FEF089596
:10359000842F0E94AC1980E00895EF92FF920F9360
:1035A0001F93CF93DF93C82FD0E0CC0FDD1FCC0F3C
:1035B000DD1FCC0FDD1FC60FD11DC05CDF4FCC0F50
:1035C000DD1FC295D295D07FDC27C07FDC27EE249B
:1035D000FF248701000F111F085B1A4FF80180813B
:1035E0009181892FBE010E94AC19F80180819181DF
:1035F0002196BE010E94AC190894E11CF11C219691
:10360000F0E1EF16F10429F7DF91CF911F910F91AF
:10361000FF90EF90089590E0880F991F8F5F934F70
:103620000E94F01990E008950F931F93082F10E067
:10363000000F111FC8018050944F0E94F01990E0B4
:10364000019609531C4FF80120813181821793079D
:1036500008F49C01C9011F910F9108958091B7044E
:1036600080937905809179050E94141B90937405CD
:1036700080937305809179050E940B1B90937B05C5
:1036800080937A0520917A0530917B0580917305AE
:10369000909174052817390720F010927B0510923D
:1036A0007A058091680590916905E0917905F0E0CF
:1036B000EE0FFF1FE953FC4F608171810E94694149
:1036C00090936905809368050895803198F470E0BF
:1036D0006050784F90E000249695879507949695D2
:1036E00087950794982F802D680F791F8CE06030A4
:1036F000780710F08FEF0895CB010E94F01908951C
:10370000EF92FF920F931F93CF93DF93E0906805A2
:10371000F09069050894E11CF11C80E00E94400FC4
:103720008823C9F400E080917C05813029F180E094
:103730000E94170F882329F080917C05882309F0C7
:10374000BFC0013009F4E7C0DF91CF911F910F9105
:10375000FF90EF90089581E080937C0510927805AA
:103760001092770580935E0482E20E94951101E039
:1037700080917C058130D9F60E945E10282F882325
:10378000B9F0215080917705909178057C01EE0C7D
:10379000FF1CEE0CFF1CEE0CFF1C880F991FE80E9F
:1037A000F91EE20EF11CF0927805E092770501E037
:1037B00087E10E94010F882341F0E0907A05F090A4
:1037C0007B050894E11CF11C01E083E00E94010FDD
:1037D000882329F0E0907305F090740501E089E0FA
:1037E0000E94010F882309F0A2C089E00E94170FF0
:1037F000882309F0BAC08AE00E94010F882309F0EB
:10380000A5C08AE00E94170F882309F490CF8CE1AD
:103810000E949511E091790520917305309174050E
:10382000F0E0EE0FFF1FE953FC4F808191812817D4
:10383000390708F07CCF809173059091740501964B
:103840009093740580937305809179056091730559
:10385000709174050E94881A809179050E94141B4A
:10386000909374058093730560917305709174054E
:10387000615070408091680590916905861797079F
:10388000D8F4EB01219701C0E901809179051C2F43
:103890006C2F0E94651B482F809179051F5F612F57
:1038A0000E94B11A9E01215030408091680590918C
:1038B00069058C179D0740F388E08093610437CF3A
:1038C00082E20E945D1110925E0410927C0581E0FC
:1038D0008093610420917705309178052115310599
:1038E000A9F0E0917905F0E0EE0FFF1FE953FC4FDE
:1038F000808191818217930748F0215030403093A6
:1039000069052093680587E080936104109236046E
:10391000013009F019CFC7010E94EB010093360472
:10392000DF91CF911F910F91FF90EF9008958BE160
:103930000E945D111092780510927705E09068055D
:10394000F09069050894E11CF11C4FCF8CE10E94B6
:103950005D111092780510927705E0906805F0905F
:1039600069050894E11CF11C4CCF8BE10E94951174
:10397000C0916805D0916905219680917305909159
:103980007405C817D90708F036CF809179051C2F28
:103990006C2F0E94651B482F809179051150612F73
:1039A0000E94B11A21968091730590917405C817F1
:1039B000D90758F3809173059091740501979093FE
:1039C00074058093730580917905609173057091FA
:1039D00074050E94881A809179050E94141B9093A7
:1039E00074058093730588E08093610404CFEF929F
:1039F000FF920F931F938091B70480937905809174
:103A000079050E94141B909374058093730580912F
:103A100079050E940B1B90937B0580937A0520917A
:103A20007A0530917B058091730590917405281774
:103A3000390720F010927B0510927A058091680575
:103A400090916905E0917905F0E0EE0FFF1FE953D1
:103A5000FC4F608171810E94694190936905809358
:103A600068058091790560916805709169050E94EB
:103A7000651B80937005809179056091700547EC16
:103A800055E02FE735E001E815E0E3E9EE2EE6E04A
:103A9000FE2E0E942B1A81E080930F060E94E424E0
:103AA0008091930680939A061F910F91FF90EF905B
:103AB0000895AF92BF92CF92DF92EF92FF920F9351
:103AC0001F93CF93DF93C82EDD24CC0CDD1CCC0CD0
:103AD000DD1CCC0CDD1CC60ED11C80E490E0C80EB1
:103AE000D91ECC0CDD1CC294D29410EFD122DC2460
:103AF000C122DC24AA24BB24C6010E94F019D82FBD
:103B0000C0E07501EE0CFF1CE8E4F5E0EE0EFF1ED0
:103B1000F701D183C08300811181C60101960E9403
:103B2000F01990E0082B192BF701118300830894FA
:103B3000A11CB11C82E090E0C80ED91E90E1A9162C
:103B4000B104D1F6DF91CF911F910F91FF90EF90CB
:103B5000DF90CF90BF90AF9008951092720584E2ED
:103B60000E9495110E940C120E94981310920D064B
:103B700080E00E94E31808951092710510920D06DE
:103B800010926A0580E00E94E3180E940C120E94C5
:103B900098130E947810089580916E0590916F059A
:103BA000682F6770969587959695879596958795D2
:103BB0008F700E945C2860916E0570916F059B016B
:103BC00040E050E0DA01C90180709078A070B070D8
:103BD000892F9A2FAB2FBB2780936804DA01C90184
:103BE00080709074A070B070892F9A2FAB2FBB2774
:103BF000809366042070307240705070232F342FF1
:103C0000452F55272093670410928205872F8F71C7
:103C100084FD806E089581E08093710581E20E94A9
:103C20005D11109266048091660480936704809110
:103C300067048093680410926A0510920D068091C3
:103C400048059091490590936F0580936E058F5FAD
:103C50009F4F89F01092760510928205109274049D
:103C60000E94CC1D8093570480912D0480FDFCCFD1
:103C700081E080936A050E942112089581E080937B
:103C8000720584E20E945D110E9421120895DF9264
:103C9000EF92FF920F931F938091F906882309F406
:103CA00081C284E00E94682510926D0580916D05A7
:103CB00080936C0510927C05109278051092770520
:103CC0000E94F71C8091AB066091EC0640910806BB
:103CD00020910E0602E516E00E941A28809108063F
:103CE00060910E064091810520910F060091850597
:103CF000E0907F050E94531457E0D52E07C0113085
:103D000009F4FBC00E948E278823C9F00E94B010DE
:103D1000109192061330D9F0143088F31430D9F191
:103D20001D3081F781E00E94002C809192068D3039
:103D300049F310926C040E948E27882339F70E9461
:103D400070270E94B01010919206133029F70E943C
:103D50006E25882309F09CC10E94E026882321F06B
:103D600010925E0410926C040E94960F882351F208
:103D7000182F11500E944113812F0E941813109385
:103D800093068091F906882309F0BCCF80919306B1
:103D900080939A06B7CF0E946E25882309F05AC1F6
:103DA00080917C05882309F44AC10E94801B83E02E
:103DB0000E94400F882309F03BC187E10E94400F19
:103DC000882309F02EC186E10E94400F882309F460
:103DD00068C080910F06882309F0AEC180919306D8
:103DE00080939A06E0906805F090690580916D05D2
:103DF000882309F08EC180910E06882309F44AC0F9
:103E000010E02091EC063091080680919A0690E02F
:103E100082959295907F9827807F98278093700550
:103E200080917005220F220F220F230F210F2F7078
:103E3000282B209370058091790560916805709119
:103E40006905409170050E94B11A1F5F8091680555
:103E5000909169050196909369058093680508948F
:103E6000E11CF11C8091680590916905E09179054C
:103E7000F0E0EE0FFF1FE953FC4F608171810E945B
:103E80006941909369058093680580910E06181723
:103E900008F4B7CF80916C05882309F050C1D09207
:103EA000610480916104873009F405C18091610447
:103EB000883009F457C180916104813009F4AEC0A3
:103EC00080919206843011F010926C048091F90672
:103ED000882309F4D9C080916B04813009F012CF96
:103EE00010926B040E94B324882309F40BCF1F9116
:103EF0000F91FF90EF90DF9008950E946E25882328
:103F000009F073C00E94801B83E00E94400F882349
:103F100039F583E00E94170F8823F1F49091790519
:103F20008091B704981711F00E94F71C80919206B7
:103F3000813011F010926C048091F906813009F4FF
:103F4000B6C00E94B324882309F4DCCE1F910F91E0
:103F5000FF90EF90DF90089583E20E949511DECFED
:103F60001092690510926805809179056091680545
:103F7000709169050E94651B809370058091790599
:103F80006091700547EC55E02FE735E001E815E05A
:103F9000A3E9EA2EA6E0FA2E0E942B1A81E0809374
:103FA0000F068091930680939A060E94E4248091E4
:103FB000AB066091EC064091080620910E0602E5E2
:103FC00016E00E941A288091080660910E06409122
:103FD000810520910F0600918505E0907F050E94E4
:103FE000531483E20E945D1194CF0E940C1282E26E
:103FF0000E945D1110936C0481E20E9495118091E2
:10400000080660910E064091810520910F060091EF
:104010000806E0907F050E94531474CF109261044B
:104020004FCF81E080936D0580E00E947911CBCE67
:1040300081E080936C0583E20E947911BECE0E94DC
:104040005D278091790586958093C10480E00E9468
:10405000002CABCE0E940C1282E20E945D1181E026
:1040600080936C0481E20E945D118091080660914A
:104070000E064091810520910F0600910806E09000
:104080007F050E9453148CCE81E00E94682523CFC7
:104090000E940C1211E010935E0484E20E945D11F4
:1040A000809193060E94181310936C0455CE84E0FF
:1040B0000E94682546CF80917905609168057091CE
:1040C00069050E94651B8093700580917905609158
:1040D000700547EC55E02FE735E001E815E093E97E
:1040E000E92E96E0F92E0E942B1A11E010930F068C
:1040F0008091080660910E064091810520910F067F
:1041000000918505E0907F050E945314109361048F
:10411000D2CE10926D05809179056E2D0E94781A8D
:10412000809179050E940B1B90937B0580937A0503
:1041300080E00E9495115FCE0E94E4244FCE109241
:104140006C0580917905B7010E94881A80917905E4
:104150000E94141B909374058093730583E20E9460
:1041600095119DCE809179056091680570916905E2
:104170000E94651B809370058091790560917005A0
:1041800047EC55E02FE735E001E815E0B3E9EB2E09
:10419000B6E0FB2E0E942B1A81E080930F0610924E
:1041A000610489CE81E00E9468257ECDEF92FF9266
:1041B0000F931F938091F906882309F4A9C184E025
:1041C0000E94682510926D0580916D0580936C05A5
:1041D00010927C0510927805109277050E94F71CCA
:1041E0008091AB066091EC064091080620910E0686
:1041F00002E516E00E941A288091080660910E06DA
:104200004091810520910F0600918505E0907F0582
:104210000E94531408C0143009F45FC00E948E2716
:10422000882309F48FC00E94B010109192061130BB
:1042300091F70E946E25882309F0D5C083E00E9483
:10424000400F882309F0F0C083E00E94170F8823F5
:1042500009F034C180E00E94400F882309F037C183
:1042600080E00E94170F882309F046C190917905DC
:104270008091B7049817E1F00E94F71C8091AB067B
:104280006091EC064091080620910E0602E516E0CA
:104290000E941A288091080660910E0640918105BF
:1042A00020910F0600918505E0907F050E94531430
:1042B00080919206813011F010926C048091F90681
:1042C000813009F421C10E94B324882309F4A6CFC8
:1042D0001F910F91FF90EF9008950E946E25882303
:1042E00009F060C086E10E94400F882309F04EC0AB
:1042F00083E00E94400F8823E9F580E00E94400F90
:10430000882319F580E00E94170F882359F58091C2
:104310009206843011F010926C048091F906882383
:1043200009F45DC080916B04813009F077CF109261
:104330006B040E94B324882359F60E948E27882399
:1043400009F071CF0E9470276ECF11E010937C05A9
:1043500082E20E9495111093360480E00E94170FAC
:104360008823A9F282E20E945D1110927C051092CE
:104370003604CDCF81E080936C0583E20E945D110D
:1043800010926D0580E00E949511B7CF81E0809377
:104390006D0580E00E945D1110926C0583E20E9421
:1043A0009511A6CF0E940C1282E20E945D1181E05D
:1043B00080936C0481E20E945D11809108066091F7
:1043C0000E064091810520910F0600910806E090AD
:1043D0007F050E94531481E00E94270283CF81E071
:1043E0000E9468259FCF0E940C1282E20E945D11FC
:1043F00010936C0481E20E949511809108066091EF
:104400000E064091810520910F0600910806E0906C
:104410007F050E94531481E00E94270283E00E94DE
:10442000400F882309F410CF109269051092680597
:104430008091790560916805709169050E94651BFE
:1044400080937005809179056091700547EC55E087
:104450002FE735E001E815E073E9E72E76E0F72E67
:104460000E942B1A81E080930F068091930680931F
:104470009A060E94E4248091AB066091EC0640917C
:10448000080620910E0602E516E00E941A28809187
:10449000080660910E064091810520910F0600915B
:1044A0008505E0907F050E94531483E20E945D1110
:1044B00083E00E94170F882309F4CCCE83E20E9488
:1044C000951180E00E94400F882309F4C9CE11E0C5
:1044D00010937C0582E20E9495118091680590916D
:1044E000690501960E94EB011093360480E00E945A
:1044F000170F882309F4BACE82E20E945D11109250
:104500007C0510923604B2CE84E00E946825DBCE92
:1045100081E00E94682556CEEF920F931F93109270
:1045200059048091F906882309F419C284E00E9495
:10453000682510926D0580916D0580936C05109231
:104540007C0510927805109277050E942E1B07C0FB
:10455000113009F48FC00E948E278823C9F00E9471
:10456000B010109192061330D9F0143088F3143043
:10457000D9F11D3081F781E00E94002C80919206D4
:104580008D3049F310926C040E948E27882339F7EE
:104590000E9470270E94B01010919206133029F7E4
:1045A0000E946E25882309F0B0C00E94E02688236F
:1045B00021F010925E0410926C040E94960F8823E2
:1045C00051F2182F11500E944113812F0E9418138D
:1045D000109393068091F906882309F0BCCF80914F
:1045E000930680939A06B7CF0E946E25882309F020
:1045F000D3C080917C05882309F4C3C083E00E9466
:10460000400F882329F080915904813009F483C137
:1046100087E10E94400F882309F08CC080E00E944F
:10462000400F882309F092C080E00E94170F882372
:1046300009F09AC080919206843011F010926C04B7
:104640008091F906882309F46FC080916B04813052
:1046500009F081CF10926B0480915904882309F0EE
:104660007ACF0E94B324882309F475CF1F910F914C
:10467000EF9008950E946E25882309F0D7C080919D
:104680007C05882309F4F7C083E00E94400F88234B
:1046900079F081E08093590480915904882309F4CA
:1046A0002EC183E20E945D11109269051092680587
:1046B00080E00E94400F882309F0E8C010917C053B
:1046C000113009F4FBC080E00E94170F882309F025
:1046D00087C0909179058091B704981711F00E94D6
:1046E0002E1B80919206813011F010926C04809103
:1046F000F906813009F0B5CF84E00E9468250E9458
:10470000B324882309F427CFB1CF0E940C1211E003
:1047100010935E0484E20E945D11809193060E94D2
:10472000181310936C0441CF81E00E946825109209
:1047300059048BCF81E080936D0580E00E94791150
:1047400080E00E94400F882309F46ECF11E010939F
:104750007C0582E20E9495111093360480E00E944D
:10476000170F882309F466CF82E20E945D11109230
:104770007C0580913604813009F4E2C01092360441
:1047800059CF0E945D278091790586958093C10459
:1047900080E00E94002C32CF0E940C1282E20E9424
:1047A0005D1181E080936C0481E20E945D11809133
:1047B000080660910E064091810520910F06009138
:1047C0000806E0907F050E945314809159048823C5
:1047D00009F499C083E20E9479110E94611309CF04
:1047E00082E20E945D1110927C0520917705309144
:1047F00078052115310591F0E0917905F0E0EE0F93
:10480000FF1FE953FC4F808191818217930730F09D
:10481000215030403093690520936805809136041B
:10482000813009F47EC01092360453CF0E940C12DE
:1048300082E20E945D1110936C0481E20E94951146
:104840008091080660910E064091810520910F0627
:1048500000910806E0907F050E945314809159044E
:10486000882309F454C083E20E945D1180917C0585
:10487000882309F009CF0E945D27809179058695EC
:104880008093C10480E00E94002CFECE11E01093C2
:104890007C05109278051092770582E20E949511AE
:1048A000809168059091690501960E94EB01109333
:1048B000360410917C05113009F005CF0E945E107E
:1048C000482F882309F4FFCE41502091770530917D
:1048D0007805C901880F991F880F991F880F991FA4
:1048E000220F331F820F931F840F911D9093780521
:1048F000809377050E94EB0110933604E4CE83E2A7
:104900000E949511D1CE83E20E94951166CF83E279
:104910000E949511B4CE80936C0583E20E945D11D4
:1049200077CE8091080660910E0640918105209116
:104930000F0600910806E0907F050E94531473CF84
:104940008091080660910E064091810520910F0626
:1049500000910806E0907F050E9453140FCF81E07C
:104960000E946825E6CD9091B6048091BC04891719
:1049700031F08091B6048093BC0481E0089580E01A
:10498000089580910F06882391F08091C705809348
:10499000AB0680917F058093EC0680918105809322
:1049A000080680910F0680930E0610920F068091E4
:1049B0000E06882329F080910E0680930E06089536
:1049C00081E080930E0608958091C7058093AB0621
:1049D00080917F058093EC06809181058093080685
:1049E00080910F0680930E0610920F060895833073
:1049F00059F0843050F0843029F0809193068093F0
:104A00009A0608951092930608958230B0F708959B
:104A1000FC0187858F708D30C1F030E020E190E09F
:104A200080818F708E3061F09F5F31969217C0F356
:104A3000892F913118F48150832B089580E1FBCFA9
:104A40009923B1F780E0832B089530E12FE0E7CF81
:104A50001F93DF93CF930F92CDB7DEB7162F0E942F
:104A60000825898389818F708F5F8093E903109374
:104A70008505898184FD08C086E08093E7030F9057
:104A8000CF91DF911F91089588E08093E7030F9005
:104A9000CF91DF911F910895E82FF0E0EF73F07050
:104AA000E651FC4F80810895409383056093C605CD
:104AB0008093920681E080930B060895882339F055
:104AC0008091C6058093920681E080930B0608953D
:104AD0008093920681E080930B06089580910B06E7
:104AE000882319F010920B0681E008953F924F92AF
:104AF0005F926F927F928F929F92AF92BF92CF926E
:104B0000DF92EF92FF920F931F93CF93DF93462E86
:104B10004A015901662309F4C4C09C01E90100E07F
:104B2000FF241FEFDD2466247724B2E05B2E3324BC
:104B30003394CE010E940825F301EA56F94F808391
:104B4000C0802FE0C222C39440E050E012C01E2576
:104B50001F7BF1F4F501E00FF11D3082FF2009F019
:104B600070C0DD24D3940F5F4F5F5F4F1E2D4C1537
:104B700088F5642FFE01E40FF51FE0802E2D30E054
:104B8000C9018F7090700F9709F455C0DD20F9F6B8
:104B9000F501E00FF11D5082EF2DF0E0D401AE0FD2
:104BA000BF1FEC926295607FE05FF94F6083F394E2
:104BB0000024220F331F001C220F331F001C232F41
:104BC000302DDD24D394D2220F5F4F5F5F4F1E2D17
:104BD0004C1578F20894611C711C6096641408F4FA
:104BE000A8CF003408F061C08F2DF501E00FF11D52
:104BF00010820F5F0034C8F39FE39F1550F09FEFC2
:104C0000EF2DF0E0E05FF94F9083F3942FE32F1541
:104C1000B8F7DF91CF911F910F91FF90EF90DF9048
:104C2000CF90BF90AF909F908F907F906F905F904C
:104C30004F903F900895F501E00FF11D1082DD24A3
:104C400092CFEF2DF0E03197E80DF91DE082FA9454
:104C5000EF2DF0E0F394E05FF94FA081AF70BA2F31
:104C6000BF5F808182958F70682F70E0CB018B0FC2
:104C7000911D40970CF0BA2F0024220F331F001C07
:104C8000220F331F001C232F302DDD24D394D2227A
:104C900062957295707F7627607F7627B62BB083FA
:104CA00062CF00E0FF2480E0A0CF8F2DA5CF2F9210
:104CB0003F924F925F926F927F928F929F92AF92AC
:104CC000BF92CF92DF92EF92FF920F931F93CF93F9
:104CD000DF935C01562E3A016901662309F45DC039
:104CE000482EEC0130E060E0EE24FF24FA9480E0EE
:104CF00000E010E05FE04EE0342E2DE0222E96E939
:104D0000892E96E0992E800E911EF40170817F709D
:104D10007F5FDE0190E0442D41950BC05C93223013
:104D200089F0E42EEA0E3F5F9F5F1196822F97175E
:104D3000D0F4F601E30FF11D2081213079F78823AB
:104D400049F45C93F301E60FF11DF0806F5FFC9274
:104D500022E0E7CF5C93F501EE0DF11D80818064C8
:104D60008083FC92DECF903158F4FE01E90FF11DF3
:104D700030829F5F05C0FE01E90FF11D50839F5FE8
:104D80009031C8F3F401808184FD2F860F5F1F4F9F
:104D90006096822F051508F4B2CFDF91CF911F9155
:104DA0000F91FF90EF90DF90CF90BF90AF909F90CA
:104DB0008F907F906F905F904F903F902F900895CD
:104DC000809183050E94170F882339F08091C605D2
:104DD0008093920681E080930B06089510927205ED
:104DE00084E20E94951110925B0480E00E9495116C
:104DF0000E9498130E949C120E9421128091C0046C
:104E00000E942F1280E00E94E318089581E08093B1
:104E1000720584E20E945D110E94211280E00E94CE
:104E20002F1280E00E94E318089510920D060E9450
:104E30009C120E9421120E9498138091C0040E942B
:104E40002F121092090681E20E94951180E00E94C3
:104E5000E3181092F9068CEF0E94DA0C0895109274
:104E6000820581E08093090681E20E945D1180E065
:104E70000E94E31880912C04882321F480912D0452
:104E800080FDFCCF10922D0410923A041092390448
:104E900010923D0410923F0410923E041092800440
:104EA000809180048093810481E080930D0680933B
:104EB000F9068AEF0E94DA0C089588E00E94400FFC
:104EC000882369F09091920688E0809383059093FF
:104ED000C60583E08093920681E080930B060895D7
:104EE00080916C04882311F480E0089581E00E9491
:104EF000400F882321F081E080936D04089581E0C4
:104F00000E94010F882381F380E00E94EB0E88232A
:104F100059F382E080936D0481E0089580912C0420
:104F2000823011F080E008950E94090D8093EE0612
:104F300080E00895EF92FF920F931F93CF93DF933A
:104F4000182F062F0E946113E12EFF24EE0CFF1C88
:104F5000EE0CFF1CEE0CFF1CE00EF11CE294F29430
:104F600050EFF522FE24E522FE24C0E0D0E0FE0151
:104F7000E556F94F8081BE016E0D7F1D0E94AC1970
:104F80002196C031D10599F70E946113DF91CF912D
:104F90001F910F91FF90EF900895CF92DF92EF92C3
:104FA000FF920F931F93CF93DF93E22E6801082F98
:104FB00010E0000F111F060F111D000F111F000F31
:104FC000111F000F111F040F111D02951295107F64
:104FD0001027007F1027FF24E294F29470EFF7224D
:104FE000FE24E722FE24FE2C82E00E945D110E9436
:104FF0006113EE2089F0C0E0D0E0F601EC0FFD1F58
:105000008081B8016C0F7D1F0E94AC1984E00E9462
:10501000470C2196CF1588F382E00E9495110E94DB
:105020006113DF91CF911F910F91FF90EF90DF906F
:10503000CF900895BF92CF92DF92EF92FF920F939D
:105040001F93CF93DF936801E82EFF24EE0CFF1C23
:10505000E60EF11CEE0CFF1CEE0CFF1CEE0CFF1C10
:10506000E40EF11CE294F29410EFF122FE24E1220E
:10507000FE2430E022953295307F3227207F322780
:10508000B22E222379F0C0E0D0E086010C0F1D1F64
:10509000C7018C0F9D1F0E94F019F8018083219693
:1050A000CB1598F3DF91CF911F910F91FF90EF9067
:1050B000DF90CF90BF900895EF92FF920F931F93D0
:1050C000CF93DF93182F062F0E946113E12EFF2448
:1050D000EE0CFF1CEE0CFF1CEE0CFF1CE00EF11C96
:1050E000E294F29490EFF922FE24E922FE24C0E03B
:1050F000D0E0CE018E0D9F1D0E94F019FE01E556F5
:10510000F94F80832196C031D10599F710925B0445
:1051100080E00E94B2110E946113DF91CF911F9134
:105120000F91FF90EF90089580912C04882349F40B
:105130000E94A50080912C04813049F00E94A00EAD
:1051400008950E94AD0380912C048130B9F70E942C
:10515000A70E08959F92AF92BF92CF92DF92EF92E7
:10516000FF920F931F9381E08093920680930B062A
:1051700000E011E0B2E0FB2EAFE0EA2EF4E0DF2E1B
:10518000E6E0CE2E77E0B72E6AE0A62E50E2952E0E
:105190000E94B01080919206863009F46FC087306B
:1051A00008F0AAC0813009F456C1843089F7809193
:1051B0000B06882339F010920B06109361041092AD
:1051C0005F0400E0809183050E94170F882331F16E
:1051D0008091C6058093920610930B060023E1F0A0
:1051E00080915F04882311F410935F0480915F0421
:1051F000813210F090925F049091000280915F04E0
:10520000981751F080915F04809300026091000232
:1052100087E090E00E945002109236040E945E10D7
:10522000282F882381F080915F048A9DC00111247A
:1052300080935F0480915F048150820F80935F04AC
:10524000F092610401E080916104882309F4A0CF09
:105250009091000280916104823009F4FDC1892F90
:1052600090E00E94EB0110933604109261040E94BA
:10527000B01080919206863009F091CF80910B0694
:10528000882339F010920B061092610410925F048B
:1052900000E0809183050E94170F882349F08091D8
:1052A000C6058093920610930B06002309F0D7C120
:1052B00080915F04882309F475C120915F04213037
:1052C00009F453C120915F04223009F422C1809176
:1052D0006104813009F43EC180916104823009F09B
:1052E00057CF109261040E942112809193040E9472
:1052F0002F120E9461134CCF873009F450C08F30B9
:1053000009F046CF80910B06882349F010920B06D6
:10531000109361048091B7048093600400E0809151
:1053200083050E94170F882349F08091C60580935A
:10533000920610930B06002309F068C10E94E40F47
:10534000882369F0982F9150933048F480918D0410
:10535000981729F090938D041093610401E08091D7
:105360008D04813009F436C180916104882309F4E9
:105370000FCF109261040E940A130E9421128091A3
:105380008D048F5F0E94AA1280918D04813009F0F4
:10539000FFCE8091900481500E942F12F9CE80910F
:1053A0000B06882321F010920B0610936104809164
:1053B00083050E94170F882351F08091C6058093C2
:1053C000920610930B068091610481FD31C10E9409
:1053D000E40F882389F0982F9150933068F48091DE
:1053E0002C04981749F090932C040E9494288091E3
:1053F000610483608093610483E00E94010F88232D
:1054000079F0809164048F5F8093640480916404D8
:10541000817080936404809161048360809361044F
:105420008091610480FFB4CE809161048E7F80936F
:1054300061040E940A1380912C048F5F0E94AA12BB
:1054400083E20E94951180916404882309F414C1B9
:105450000E9461139DCE80910B06882331F010923B
:105460000B060E940C120E94611387E10E94400FFC
:10547000882359F09091920687E180938305909359
:10548000C605B092920610930B0688E00E94400F6A
:10549000882359F09091920688E080938305909339
:1054A000C605C092920610930B0681E00E94400F41
:1054B000882351F080919206109383058093C6054E
:1054C000D092920610930B068EE00E94400F882324
:1054D00059F0909192068EE0809383059093C605D3
:1054E000E092920610930B069091B6048091BC0452
:1054F000891709F44DCE8091B6048093BC041F91A6
:105500000F91FF90EF90DF90CF90BF90AF909F9062
:1055100008959091B70480916004981759F0809194
:10552000B7048093600420936104809160048093A9
:10553000930401E089E00E94170F882309F4C7CE85
:1055400010925F048BE10E9495118091610481307B
:1055500009F0C2CE109261040E942112809194043D
:105560000E942F120E94611313CE9091B704809174
:105570006004981759F08091B704809360042093D9
:105580006104809160048093940401E08AE00E94A9
:10559000170F882309F496CE10925F048CE10E94C5
:1055A000951190CE8AE00E94010F882309F068C00F
:1055B00089E00E94010F882309F47FCE8BE10E94CD
:1055C0005D11F0925F04F09261048091B7048093C2
:1055D000600473CE909160048091B704981709F429
:1055E000C3CE8091B70480936004909160049F5F64
:1055F000923008F451C080919004981709F4B4CE09
:10560000909390041093610401E0AECE80919004D9
:1056100060918D0490E0019782959295907F9827F4
:10562000807F9827682B8AE090E00E94500286CE07
:105630008091640490E08170907082959295907F43
:105640009827807F982760912C046F70682B82E0E8
:1056500090E00E945002BBCE90915F0400CE83E0A8
:1056600090E0609194040E94500284E090E0609188
:1056700093040E9450021CCE83E20E945D11E8CE8A
:105680008CE10E945D1110935F041093610480917E
:10569000B704809360048CCF92E0ADCF1F93DF936B
:1056A000CF930F92CDB7DEB71092F90680E00E943B
:1056B000E3188CEF0E94DA0C80912C04813011F0F9
:1056C0000E94760E80910F06882391F08091C70585
:1056D0008093AB0680917F058093EC0680918105D5
:1056E0008093080680910F0680930E0610920F0695
:1056F00090917F058091EC06981721F080917F05AD
:105700008093EC06109250061092800480918004E1
:10571000809381041092800582E596E0909395062F
:1057200080939406109108060E9408258983898138
:105730008F708F5F8093E90310938505898184FDC5
:1057400008C086E08093E7030F90CF91DF911F910F
:10575000089588E08093E7030F90CF91DF911F9128
:1057600008951F93DF93CF930F92CDB7DEB780E0FC
:105770000E94E3181092500610922D0410923A04E1
:105780001092390410923D0410923F0410923E048E
:1057900010926E04109280048091800480938104A2
:1057A0001092800582E596E090939506809394068A
:1057B000109108060E940825898389818F708F5F68
:1057C0008093E90310938505898184FD17C086E0E5
:1057D0008093E70381E08093F9068AEF0E94DA0C58
:1057E00080912C04813011F00E94740E83E080932C
:1057F00034040F90CF91DF911F91089588E0E8CF96
:10580000EF920F931F93982F882309F495C081304E
:1058100029F080E01F910F91EF90089580910B0681
:10582000882309F0F9C00E94E40F882399F1982F8A
:10583000915080910F06882341F48091080680934F
:1058400081058091AB068093C705809181058917FA
:1058500070F480918105981B9F5F90930F06809153
:105860000F06853008F446C184E080930F068091CE
:10587000F906882309F441C18091080660910E065B
:105880004091810520910F0600918505E0907F05EC
:105890000E94531484E10E94010F882309F0DEC0A6
:1058A00085E10E94010F882309F0CEC08091F9069E
:1058B000882321F59091EC0680917F059817F1F0EF
:1058C00080917F058093EC068091AB066091EC0699
:1058D0004091080620910E0602E516E00E941A2863
:1058E0008091080660910E064091810520910F0677
:1058F00000918505E0907F050E9453148091F90680
:10590000882329F480910F06882309F0D4C00E94CF
:10591000FE0F982F882309F47CCF80915F0491506B
:10592000981709F076CF8091C6058093920681E0A2
:1059300080930B0680E06ECF0E94E40F982F88239F
:10594000D1F584E10E94010F882309F49FC01092D1
:105950007F0588E00E945D1181E00E949511809191
:10596000F906882309F055CF9091EC0680917F05C8
:10597000981709F44ECF80917F058093EC068091B3
:10598000AB066091EC064091080620910E0602E5F8
:1059900016E00E941A288091080660910E06409138
:1059A000810520910F0600918505E0907F050E94FA
:1059B000531480E02FCF8091C1048093C70501E08C
:1059C00000930F06192F11501093810584E10E9456
:1059D000EB0E882309F44BC010927F0588E00E94EB
:1059E0005D1181E00E94951110935F0480919206F1
:1059F0008093C6058DE08093920681E080930B062C
:105A0000109293068091F906882309F44FC081E033
:105A10001F910F91EF90089510920B0690936C04D4
:105A20008091080660910E064091810520910F0635
:105A300000918505E0907F050E9453140E94E40FB9
:105A4000882309F427CFF3CE81E080937F0588E097
:105A50000E94951181E00E945D1128CF10927F0570
:105A600088E00E945D1181E00E94951119CF85E1C7
:105A70000E94EB0E882309F4B7CF00937F0588E0DE
:105A80000E94951181E00E945D11AECF85E10E94D8
:105A9000010F882309F463CF81E080937F0588E0BC
:105AA0000E94951181E00E945D1159CF82E00E9411
:105AB000F72481E0ADCF8091C7058093AB0680913C
:105AC0007F058093EC068091810580930806809184
:105AD0000F0680930E0610920F068091AB06609120
:105AE000EC064091080620910E0602E516E00E94A1
:105AF0001A280DCF80910F06B8CE8091C7058093EC
:105B0000AB0680917F058093EC06809181058093A0
:105B1000080680910F0680930E0610920F06809162
:105B2000AB066091EC064091080620910E0602E556
:105B300016E00E941A28A0CE2F923F924F925F92B9
:105B40006F927F928F929F92AF92BF92CF92DF928D
:105B5000EF92FF920F931F93DF93CF930F92CDB7E6
:105B6000DEB70E94B0101092930680919306809346
:105B70009A068091F906882311F40C942C3784E05E
:105B80008093920681E080930B06662499248824F2
:105B900055247724739438E0432E26E0322E93E088
:105BA000292E0E94B010109192061830D9F01930A9
:105BB00008F04CC0153009F49AC4163008F096C0AD
:105BC000113009F431C2143009F408C40E948E2740
:105BD000882339F70E9470270E94B0101091920616
:105BE000183029F780910B06882349F010920B0694
:105BF0000E940C1283E20E945D1170925E048091FB
:105C000083050E94170F8823A1F08091C605809319
:105C1000920670920B0610925E048091AB06609122
:105C2000EC064091080620910E0602E516E00E945F
:105C30001A280E94E40F882309F00BC50E94FE0F6A
:105C4000882321F281500E944B14C0CF1B3009F4ED
:105C5000DAC21C30D0F5193009F481C21A3009F0CB
:105C6000B5CF80910B068823F9F010920B0680E0E7
:105C70000E945D110E9461138091AB066091EC0659
:105C80004091080620910E0602E516E00E94CD27FD
:105C900080E00E9495110E94611384E08093920637
:105CA00070920B0610925E0480916104882339F093
:105CB00084E08093920670920B06109261048091AA
:105CC00061048F5F8093610481CF1C3009F47CC133
:105CD0001D3009F07BCF81E00E94002C809192065C
:105CE0008D3009F473CF10926C0470CF163009F424
:105CF000FCC0173009F06ACF80910B06882389F128
:105D000010920B060E940C1260910E0682E596E03E
:105D10004CEA56E026E835E00E94762580E00E94B5
:105D20005D111092610489E080935F041092600419
:105D300080910E06882391F020E0E22FF0E0EA56F1
:105D4000F94F9081809160048F5F9F70890F8093DD
:105D500060042F5F80910E06281778F3662499243B
:105D6000552480E00E94400F882311F0662463943C
:105D700088E00E94400F882311F012E0612E87E135
:105D80000E94400F882311F0B3E06B2E80915F04D6
:105D9000893009F420C680915F04813009F4F5C58B
:105DA00080915F04882309F491C580915F04882362
:105DB00029F080915F04807F09F45FC010915F0437
:105DC0008EE00E94010F882351F080915F04806172
:105DD00080935F0485E080936104F2E05F2E8FE0A2
:105DE0000E94010F882351F080915F0480628093AC
:105DF0005F0485E0809361045524539484E10E94FC
:105E0000010F882349F080915F04806480935F04D0
:105E100085E08093610455248EE00E94170F88234B
:105E200041F080915F04807E80935F0484E08093E2
:105E300061048FE00E94170F882341F080915F0476
:105E4000807D80935F0484E08093610484E10E94FC
:105E5000170F882341F080915F04807B80935F045B
:105E600084E08093610480916104853009F462C507
:105E700080916104843009F44DC580915F048830BD
:105E800009F413C58091610490E083709070892BB0
:105E900009F03BC4662009F499CE60910E0682E5B4
:105EA00096E04CEA56E026E835E00E9457268091BD
:105EB000AB066091EC064091080620910E0602E5C3
:105EC00016E00E94CD2791E0691609F446C5E2E08C
:105ED0006E1609F474C0F3E06F1609F077CE87E010
:105EE0008093920670920B0671CE80910B068823E8
:105EF000D9F010920B060E940C1260910E0682E5FA
:105F000096E04CEA56E026E835E00E94762584E2E9
:105F10000E945D111092610410926004E3E6E09328
:105F20005F0466249924882480E00E94400F88231F
:105F300011F06624639488E00E94400F882311F0DA
:105F400082E0682E80915F04833609F403C6809155
:105F50005F04813009F49FC580915F04833009F4A8
:105F600045C580915F04882309F440C48091610491
:105F700090E083709070892B09F008C4662009F4C2
:105F800025CE60910E0682E596E04CEA56E026E8C2
:105F900035E00E9457268091AB066091EC06409157
:105FA000080620910E0602E516E00E94CD2791E03A
:105FB000691609F4D2C4E2E06E1609F007CE3092F9
:105FC000920670920B0602CE80910B06882389F010
:105FD00010920B0690915C0480910E06981709F4BC
:105FE000F7C5709261048091C60580939206709205
:105FF0000B06809183050E94170F882309F4E6CDD4
:106000008091C6058093920670920B068091610480
:10601000882309F4F0C58DE00E94951182E00E946A
:1060200095110E946113D2CD80910B068823E9F06F
:1060300010920B0680E00E9427020E940C1282E25E
:106040000E945D1110936C0481E20E949511809171
:10605000080660910E064091810520910F0600917F
:106060000806E0907F050E94531480E00E94002CF7
:1060700080E00E94010F882329F085E0809392063A
:1060800070920B0683E00E94010F882351F08091EB
:106090009206209283058093C605409292067092E4
:1060A0000B0688E00E94400F882321F03092920670
:1060B00070920B0687E10E94400F882329F087E049
:1060C0008093920670920B068BE00E94400F88230B
:1060D00059F0909192068BE0809383059093C605CA
:1060E0008093920670920B068DE00E94400F8823E9
:1060F00061F0909192068DE0809383059093C605A0
:106100009CE09093920670920B06809192068130EB
:1061100011F010926C049091F906913009F4C8C204
:106120009091B6048091BC04891709F44FCD8091F9
:10613000B6048093BC040F90CF91DF911F910F9113
:10614000FF90EF90DF90CF90BF90AF909F908F9097
:106150007F906F905F904F903F902F900895809127
:106160000B06882371F010920B0682E20E949511B3
:1061700081E00E94E31880E00E94E31880E00E9422
:10618000270290915F04809184059817C9F0909040
:106190005F048091840580935F0480916104833063
:1061A00009F4A6C580916104823050F080917E058B
:1061B000882331F4E0915F04F0E0EA57FA4F7082EF
:1061C00086E10E94010F882329F080917E058823B3
:1061D00009F4CBC480916104833009F4C3C386E120
:1061E0000E94170F882309F4F1CC8091610482305A
:1061F00009F0ECCC7092610480E00E94E31882E028
:106200000E949511E3CC80910B06882361F01092D7
:106210000B0682E20E9495118FE00E945D110E94A0
:10622000611310926104809183050E94170F8823E7
:1062300009F442C08091C6058093920670920B06C5
:1062400080916104882391F58091AB063091EC0632
:106250002091080690E0880F991F830F911D880FE9
:10626000991F880F991F880F991F280F20935D048D
:1062700080910E0680935C048823C1F090E0A0E03A
:10628000B0E0282F30E022953295307F3227207FF2
:106290003227FD01EE5AF94F8081A853BA4F8C93F3
:1062A0009F5FA92FB0E0A217B3079CF38FE00E9475
:1062B00095118DE00E9495118DE00E94010F8823B9
:1062C00009F484CC80916104882309F07FCC80910B
:1062D0005C04882309F47ACC709261048091AB0647
:1062E0002091EC061091080690E0880F991F820F0C
:1062F000911D880F991F880F991F880F991F180FDC
:1063000080915D04181709F461CC8DE00E945D1145
:1063100082E00E945D110E94611360915D04809192
:106320000E06882309F440C0C62EDD24C294D29400
:10633000E0EFDE22DC24CE22DC24A12EBB24A294BA
:10634000B29470EFB722BA24A722BA24750100E0F4
:1063500010E0C6010E94F019882E0E5A194FF8015C
:106360008083C7010E94F019B6010E94AC19882DE4
:10637000B7010E94AC1984E00E94470C0894C11C2C
:10638000D11C0894E11CF11C8E2D8A19082F10E0F5
:1063900080910E0690E082959295907F9827807F5D
:1063A000982708171907ACF21091080682E596E0C5
:1063B0000E940825898389818F708F5F8093E9030C
:1063C00010938505898184FD51C586E08093E7039C
:1063D00082E00E9495110E946113F8CB80910B0618
:1063E0008823E9F010920B060E940C1282E20E94B0
:1063F0005D1170926C0481E20E945D11809108062B
:1064000060910E064091810520910F0600910806CB
:10641000E0907F050E94531481E00E94270283E0F0
:106420000E94400F882309F445C080910F068823FD
:1064300009F03CC49091EC0680917F05981781F09B
:1064400080917F058093EC068091AB066091EC060D
:106450004091080620910E0602E516E00E941A28D7
:1064600060910E0682E596E04CEA56E026E835E0BB
:106470000E94762580E090E0FC01EA57FA4F1082F6
:10648000019680349105C1F782E080935E041092FA
:10649000EF061092600410925F0410926104109253
:1064A0007E057092630489E08093920670920B06D9
:1064B00099249A9480919206843011F010926C0481
:1064C0008091F906882321F47092920670920B064F
:1064D00080916B04813009F079CB10926B0490911C
:1064E000B6048091BC04891709F021CE6FCB80914E
:1064F0000B068823C9F010920B060E940C127092B2
:10650000610482E596E00E940825282F2F702F5FF6
:1065100020935F0490E0929582958F7089279F70F9
:1065200089278170809360048EE00E947F10823002
:1065300009F4DEC08AE00E947F10823009F4BEC0F8
:1065400089E00E947F10823009F4C6C08FE00E946B
:10655000010F882399F020926104809160048823C0
:1065600019F49CE090935F04809160048F5F8093A6
:106570006004809160048170809360048091610464
:1065800080FF21C0809161048150809361048091DB
:106590006004882309F4ABC180915F04803108F462
:1065A000A1C381E080935F0483E00E945D1180912C
:1065B0005F04882309F0ABC181E080935F04809180
:1065C0005F040E943A1280E00E94170F882309F4AA
:1065D000FDCA809161048230B8F182E080935E044C
:1065E00082E596E061E04CEA56E026E835E00E945C
:1065F000762590915F0480916004811180E1915033
:106600009F70892B8093960682E596E061E04CEAC4
:1066100056E026E835E00E9457268091AB0660914F
:10662000EC064091080621E002E516E00E94CD2725
:106630008091AB066091EC064091080620910E0611
:106640000E941A2810925E047092920670920B06B5
:10665000BDCA182F1150812F0E9443148091AB06A0
:106660009091EC06E82EFF24EE0CFF1CE90EF11CC5
:10667000EE0CFF1CEE0CFF1CEE0CFF1CE10EF11CDF
:10668000E294F29450EFF522FE24E522FE248701E5
:10669000005F1F4F8FE0B7010E94AC1984E00E9499
:1066A000470C0894E11CF11CE016F10699F7C6CAE4
:1066B00084E08093920690930B0632CD80915F0424
:1066C0008F708F5F80935F042092610489E00E9445
:1066D0007F10823009F03ACF80915F0490E00E96EF
:1066E0008F7090708F5F80935F04209261042ECF33
:1066F00080916104823008F477C380915F048F5FDA
:1067000080935F042092610415CF0E942112809132
:106710000E068823B1F090E080E001C08E2FE92FB3
:10672000F0E0EA56F94FE081EF70EF5FE80F98165E
:1067300018F09E1608F4E5C29F5F80910E06981728
:1067400068F384E00E94951183E00E94951188E02F
:106750000E9495118091610480FD13C0F2E05F16E4
:1067600009F486C381E0581609F486C3552031F038
:1067700084E00E945D1183E00E945D1188E00E9428
:106780005D110E9461131092610484CB0E9421125A
:10679000E92DF0E0E05FF94F80818F3FD1F010816B
:1067A00012951F7000810F70010F0F5F101738F0E6
:1067B00010C0812F0E9458121F5F101750F4809153
:1067C000610480FDF6CF812F0E942F121F5F1017EA
:1067D000B0F38091610480FF09C2882D60E00E94BF
:1067E000AE14109261040E946113C8CB86E10E942E
:1067F000010F882309F08FC20E94960F882309F0A9
:10680000C1C287E10E94170F882329F08FE3980EF9
:106810009822709261048EE00E94010F882321F07B
:1068200090E1892A709261048FE00E94010F882311
:1068300021F0E0E28E2A7092610484E10E94010F4F
:10684000882321F0F0E88F2A7092610485E10E948C
:10685000010F882321F080E4882A709261048EE081
:106860000E94170F882321F09FEE89227092610405
:106870008FE00E94170F882321F0EFED8E22709297
:10688000610484E10E94170F882321F0FFE78F2223
:106890007092610485E10E94170F882309F466CB8A
:1068A0008FEB88227092610461CBE92DF0E0EA570A
:1068B000FA4F5082939480916004981610F06624E9
:1068C00063947092610410925F04DCCA86E10E94B6
:1068D000400F882309F469CAE92DF0E0EA57FA4F1E
:1068E000508070925F0482E0809361045ECA809160
:1068F0005F04813108F4F9C181E080935F0483E093
:106900000E94951180915F04882309F455CE8091EF
:106910005F0453CE112359F080915F04882339F42A
:10692000939480916004981610F06624639470929A
:106930006104A3CA112309F0CCC180915F048823AC
:1069400009F4C7C1662029F4E92DF0E0EA57FA4FAF
:10695000508282E0809361048BCA609292066092BA
:106960000B0634C90E942E10882309F438CC82E02B
:106970008093610486E10E94EB0E882309F02FCCFE
:10698000709261040E94E3182ACC86E10E94170FDE
:10699000882311F040925F048EE00E94010F88234B
:1069A00029F082E080936104A2E05A2E8FE00E94D9
:1069B000010F882329F082E08093610455245394C9
:1069C00084E10E94010F882309F4EAC982E08093E0
:1069D00061045524E5C987E10E94170F882309F453
:1069E000DAC910925F0470926104D5C90E94960FB3
:1069F000182F0E94B00F882319F4112309F4B1CA8B
:106A0000E92DF0E0E455F94F808280E00E94E31820
:106A100085E00E94470C93949FE3991518F4109217
:106A2000600499247092610410925F04112309F4A8
:106A300098CA812E8A94EFE08E228EE00E94EB0E9F
:106A4000882311F0F0E18F2A8FE00E94EB0E88235B
:106A500011F080E2882A84E10E94EB0E882311F075
:106A600090E8892A85E10E94EB0E882311F0E0E48A
:106A70008E2AE82DF0E0EF73F070E651FC4F482DC0
:106A80004078808160E00E94CC1882E080936104AD
:106A900020925F0466CA86E10E94170F882309F0DE
:106AA000A8C18EE00E94010F882349F0882D8095AF
:106AB0008071FFEE8F22882A82E0809361048FE04C
:106AC0000E94010F882349F0882D809580729FEDE8
:106AD0008922882A82E08093610484E10E94010F68
:106AE000882349F0882D80958078EFE78E22882AC8
:106AF00082E08093610485E10E94010F882349F0C0
:106B0000882D80958074FFEB8F22882A82E0809305
:106B100061040E94960F182F882309F41DCA80E093
:106B20000E94E31885E00E94470C11501F7080EF0F
:106B30008822812AE82DF0E0EF73F070E651FC4FD7
:106B4000482D4078808160E00E94CC1882E08093DC
:106B5000610402CA88E00E94170F882309F4F7C96C
:106B600010925F0470926104F2C982E08093610424
:106B70000E941810882311F020926104E0915F04B4
:106B8000F0E0EA57FA4F82E08083E0916004F0E0A1
:106B9000E455F94F808080920C06E82DF0E0EF7309
:106BA000F070E651FC4F482D4078808160E00E94F3
:106BB000CC1880915F04981639F090905F04809112
:106BC00060048F5F8093600482E00E945D1102CBBD
:106BD000992309F406CA82E20E9495118DE00E9471
:106BE0005D110E9461131092610403CA882D61E057
:106BF0000E94AE14F6CD82E00E945D110E946113E6
:106C00009091AB062091EC063091080680915C04CF
:106C10008823B9F1E92EFF24EE0CFF1CE20EF11CD3
:106C2000EE0CFF1CEE0CFF1CEE0CFF1CE30EF11C27
:106C3000E294F29430EFF322FE24E322FE24870153
:106C4000A0E0B0E0FD01E853FA4F8081AE5AB94FA1
:106C50008C93B8010E94AC1984E00E94470C0F5F2E
:106C60001F4F802F8E19A82FB0E080915C0490E018
:106C700082959295907F9827807F9827A817B907CB
:106C80000CF31091080682E596E00E94082589839E
:106C900089818F708F5F8093E903109385058981C7
:106CA00084FDA5C086E08093E703B5C98091C70540
:106CB0008093AB0680917F058093EC0680918105DF
:106CC0008093080680910F0680930E0610920F069F
:106CD000BBCB939480916004981608F433CE66245D
:106CE000639437CE80915F045DCC80915F0405CEC4
:106CF0000E941810882309F055CA82E0809361042D
:106D000051CA992D981B8091610480FFA1C0892FE1
:106D10000E94581216CDE92DF0E0E455F94F80801D
:106D20008EE00E94EB0E882311F0F0E18F2A8FE0B5
:106D30000E94EB0E882311F080E2882A84E10E94F1
:106D4000EB0E882311F090E8892A85E10E94EB0E72
:106D5000882311F0E0E48E2AE82DF0E0EF73F07064
:106D6000E651FC4F482D4078808160E00E94CC18AD
:106D700082E08093610470925F040E94960F8823E2
:106D800009F43FCD882E8A94FFE08F228EE00E9486
:106D9000EB0E882311F080E1882A8FE00E94EB0E31
:106DA000882311F090E2892A84E10E94EB0E882367
:106DB00011F0E0E88E2A85E10E94EB0E882311F0A5
:106DC000F0E48F2AE82DF0E0EF73F070E651FC4F0D
:106DD000482D4078808160E00E94CC1882E080934A
:106DE000610420925F040DCD10925F0486CC88E090
:106DF0005ACFE92DF0E0E455F94F80828EE00E94F1
:106E0000EB0E882381F588248FE00E94EB0E882307
:106E100011F0F0E28F2A84E10E94EB0E882311F03A
:106E200080E8882A85E10E94EB0E882311F090E427
:106E3000892A80E00E94E3189394EFE3E91518F49F
:106E40001092600499247092610410925F0429CE1C
:106E5000892F0E942F1275CC81E080939206809337
:106E60000B060C94C52D00E1802ECECF88E0AECA73
:106E700084E00E945D1185CC83E00E945D1181CC8D
:106E80000F931F93CF93DF93EC01442319F18B01F0
:106E900050E070E020E030E0F901EA56F94F6081FF
:106EA0006F706F5FD80190E0FE01E50FF11D8081EA
:106EB0008D939F5F5F5F9617B8F3760F2F5F3F4FFD
:106EC000005F1F4F241740F3872FDF91CF911F9151
:106ED0000F91089570E0872FDF91CF911F910F914F
:106EE0000895BF92CF92DF92EF92FF920F931F937C
:106EF000CF93DF936B01B42E442369F17C0110E042
:106F000000E0C0E0D0E0C7010E940825FE01EA567B
:106F1000F94F808320812F702F5FD70190E08D91F2
:106F2000F601E10FF11D80839F5F1F5F9217B8F399
:106F3000020F219680E190E0E80EF91ECB1518F3C0
:106F4000802FDF91CF911F910F91FF90EF90DF90F5
:106F5000CF90BF90089500E0F3CFCF92DF92EF92F1
:106F6000FF920F931F93DF93CF93CDB7DEB7C0543B
:106F7000D0400FB6F894DEBF0FBECDBF10926104B3
:106F800010925F0482E080935E0440910E0682E5D9
:106F900096E06E010894C11CD11CB6010E947137A5
:106FA000E82E809160048E1510F01092600480919C
:106FB0000E068823C1F090E030E0E32FF0E0EA56BF
:106FC000F94F20812F702F5F80E0E92FF0E0E05F24
:106FD000F94F80838F5F9F5F8217B8F33F5F809187
:106FE0000E06381750F30E94B0108091F9068823DE
:106FF00009F4C5C184E00E946825FF240E94B010F6
:1070000010919206113071F01430E1F10E948E2738
:107010008823A1F70E9470270E94B0101091920659
:10702000113091F70E946E25882309F0F4C086E1A3
:107030000E94400F882329F080916204882309F080
:1070400088C180919206813011F010926C04809179
:10705000F906813009F475C10E94B3248823B1F286
:1070600010925E04C05CDF4F0FB6F894DEBF0FBE17
:10707000CDBFCF91DF911F910F91FF90EF90DF90E7
:10708000CF9008950E946E25882309F037C110E043
:1070900086E10E94400F882309F0D0C087E10E945A
:1070A000400F882309F0E6C086E10E94170F88236D
:1070B00009F0FCC087E10E94170F882309F001C185
:1070C00086E10E94010F882309F006C18EE00E942C
:1070D000010F882339F08F2D809580719FEEF92262
:1070E000F82A12E08FE00E94010F882339F08F2DDB
:1070F000809580729FEDF922F82A12E084E10E94C7
:10710000010F882339F08F2D809580789FE7F92231
:10711000F82A12E085E10E94010F882339F08F2DB3
:10712000809580749FEBF922F82A12E00E94960F56
:10713000282F882361F08F2D90E08F7090700D972D
:1071400034F421502F7080EFF822F22A12E088E008
:107150000E94010F882309F44AC08F2D90E08F70A0
:1071600090700D970CF4E8C090EFF92200E010E069
:1071700080916004F601E80FF11DF08240910E0647
:10718000C60162E576E00E944037E82E81E08093F8
:1071900062040D301105BCF58F2D61E00E94AE1424
:1071A00084E20E945D110E942112E0916004F0E0EF
:1071B000E05FF94F80810E942F120E94611380913D
:1071C0009206843011F010926C048091F9068823A5
:1071D00009F4AEC080916B04813009F017CF109292
:1071E0006B040E94B324882309F410CF39CF1230E6
:1071F00009F4C9C0113019F70F2D10E00F7010708D
:107200000D3011054CF28F2D60E00E94AE1484E227
:107210000E949511C8CF0E940C1282E20E945D115B
:1072200010936C0481E20E9495118091620488237E
:1072300009F4A1C082E00E947911F9CE8091600426
:107240008F5F80936004809160046E2D0E945D4189
:107250009093600480916004F601E80FF11DF080C6
:1072600082E00E945D1111E087E10E94400F8823B7
:1072700009F41ACF809160046E2D70E090E00197C0
:10728000860F971F0E947D41809360048091600467
:10729000F601E80FF11DF08080E00E945D1111E021
:1072A00086E10E94170F882309F404CF82E00E9430
:1072B00095110E94611387E10E94170F882309F43A
:1072C000FFCE80E00E9495110E94611386E10E942A
:1072D000010F882309F4FACE80E00E94EB0E882388
:1072E00009F4F4CE80918405809360048091600459
:1072F000F601E80FF11DF08011E0E8CE0E940C12BB
:1073000082E20E945D1181E080936C0481E20E9420
:107310005D11809162048823C1F082E00E9479119E
:1073200080916004F601E80FF11DF08011E0B0CE0D
:1073300081E00E9468254ECF8FE0F82E0FE010E02C
:1073400017CF84E00E94682587CE82E00E949511C5
:10735000E7CF82E00E9495118091AB066091EC0628
:107360004091080620910E0602E516E00E94CD2706
:107370001092620466CE82E00E94951158CE81E0A0
:107380000E9468253ACE0F2D10E00F701070F0CEDD
:107390003F924F925F926F927F928F929F92AF92A5
:1073A000BF92CF92DF92EF92FF920F931F93DF93E2
:1073B000CF93CDB7DEB7C058D0400FB6F894DEBF3C
:1073C0000FBECDBF1092610410925F0482E08093E3
:1073D0005E0440910E06B1E4CB2ED12CCC0EDD1E06
:1073E00082E596E0B6010E947137E82E0E94B01047
:1073F0008091F906882309F42CC684E00E94682550
:107400009924442488245524AA24AA94BB243324F0
:1074100033943E010894611C711C0E94B0101091BD
:1074200092061F30A9F0103108F088C0113009F41D
:10743000B8C2143009F44CC20E948E27882369F721
:107440000E9470270E94B010109192061F3059F7C9
:107450000E946E25882309F09BC40E94E02686E1E5
:107460000E94010F882309F08AC489E00E94010F5D
:10747000882309F0D5C28AE00E94010F882309F011
:10748000C7C286E10E94170F882309F0BDC289E0B8
:107490000E94170F882309F0B3C28AE00E94170FD9
:1074A000882309F0A9C28DE00E94010F882329F0EA
:1074B00080915C04882309F031C591E0991609F4A4
:1074C000DBC3A2E09A1609F4D3C3B3E09B1609F01C
:1074D000B3CF30926204682D70E0842D992787FD28
:1074E0009095860F971F850D911D0E947D41582E06
:1074F000EE2099F020E030E0F601E20FF31F852D39
:10750000820F682D0E945D41D301A90FB11D8C919E
:1075100080832F5F3F4F2E1578F340910E06C601F2
:1075200062E576E00E94403740910E0682E596E0E3
:10753000B6010E947137E82E99247ECF113109F4EB
:107540001BC1113108F480C0123109F075CF0E94BF
:107550006E25882309F056C40E94E0268CE00E9424
:10756000010F882309F077C38CE00E94170F88234E
:1075700009F06DC38EE00E94010F882309F05DC3FE
:107580008FE00E94010F882309F04DC384E10E941F
:10759000010F882309F03DC385E10E94010F882374
:1075A00009F02DC388E00E94010F882309F01DC354
:1075B0008EE00E94170F882309F0EFC28FE00E942F
:1075C000170F882309F0F2C284E10E94170F882365
:1075D00009F0F5C285E10E94170F882309F0F8C26F
:1075E00088E00E94170F882309F0FBC2992009F454
:1075F00023CF30926204EE2009F48FCF860110C0B1
:107600000E97F9F08F2D8A21D8019C919B21892B0F
:10761000F80181938F018E2F8C198E1508F07DCF84
:107620000E94E000F82E90E08F7090708D309105F0
:1076300039F7E7EFFE228F2D90E08F7090700E9754
:1076400009F7F7EFFF22DECF0E946E25882309F0AD
:107650009EC20E94E0268CE00E94010F882309F060
:10766000E7C187E10E94010F882309F0ECC180E0A7
:107670000E94010F882309F0F1C18CE00E94170FCE
:10768000882309F0F6C187E10E94170F882309F0CB
:10769000F9C180E00E94170F882309F0FCC18EE039
:1076A0000E94010F882309F0FFC18FE00E94010FA3
:1076B000882309F008C284E10E94010F882309F0A1
:1076C00011C285E10E94010F882309F01AC288E0E7
:1076D0000E94010F882309F023C28EE00E94170F39
:1076E000882309F02CC28FE00E94170F882309F02D
:1076F0002FC284E10E94170F882309F032C285E16E
:107700000E94170F882309F035C288E00E94170FE6
:10771000882309F038C2992009F48ECE3092620491
:10772000E2E09E1609F4D0C3F4E09F1609F446C4C3
:10773000B1E09B1609F003C4EE2009F4EECE8601F9
:1077400007C00F5F1F4F802F8C198E1508F0E5CEF4
:107750000E94E000F82EEFE1E81798F30E94E000A5
:10776000D8012C916E2D0E945D41F601E90FF11DAB
:1077700080818C932083E5CF0E946E25882309F0B9
:10778000F9C20E94E0268CE00E94010F882309F0D4
:10779000E8C28CE00E94170F882309F0DEC28EE059
:1077A0000E94010F882309F0CEC28FE00E94010FD2
:1077B000882309F0BEC284E10E94010F882309F0EA
:1077C000AEC285E10E94010F882309F09EC288E0C5
:1077D0000E94010F882309F08EC28EE00E94170FCD
:1077E000882309F084C28FE00E94170F882309F0D4
:1077F0005FC284E10E94170F882309F062C285E10D
:107800000E94170F882309F065C288E00E94170FB5
:10781000882309F068C28DE00E94010F882329F0B7
:1078200080915C04882309F043C0192D10FF04CE19
:107830003092620411FDEBC2EE2041F1860106C0D8
:107840000F5F1F4F802F8C198E1500F50E94E000EE
:10785000F82EBFE3B817A0F30E94E000F82E90E0E6
:107860008F7090708D30910509F400C30E9709F464
:10787000FAC29F2D9A21D8018C918B21982B9C9331
:107880000F5F1F4F802F8C198E1500F3BEEF9B22C8
:1078900040910E06C60162E576E00E9440374091B5
:1078A0000E0682E596E0B6010E947137E82EC4CD3F
:1078B000892D80958270B1E09B22982A8DE00E94EC
:1078C0009511192D91FCA2C388240E946113AECF9B
:1078D0000E946E25882309F07FC284E00E94400F39
:1078E000882309F072C285E00E94400F882309F0C6
:1078F00065C282E10E94400F882309F058C281E1ED
:107900000E94400F882309F04BC286E10E94400F7D
:10791000882329F080916204882309F0E9C287E175
:107920000E94400F882329F080916204882309F087
:10793000B2C280919206843041F010926C0482E0D1
:107940000E94951182E20E9495118091F906882388
:1079500009F48AC180916B04813009F06DCD1092D9
:107960006B040E94B324882309F466CD10925E0450
:10797000C058DF4F0FB6F894DEBF0FBECDBFCF911A
:10798000DF911F910F91FF90EF90DF90CF90BF900C
:10799000AF909F908F907F906F905F904F903F90AF
:1079A00008950E946E25882389F480919206813083
:1079B00011F010926C048091F906813009F467C2CD
:1079C0000E94B324882309F437CDD0CF0E940C1233
:1079D00082E20E945D1110936C0481E20E94951175
:1079E00080916204882309F4A6C282E00E94791182
:1079F00081E00E942702D9CF8CE10E94951153CDDE
:107A00008BE10E94951149CD82E00E9495113FCDF6
:107A10008CE10E945D119F2C93944424439431CDBA
:107A20008BE10E945D119F2C939444244A9423CDB2
:107A30008EE00E945D119924939487E10E94010FCA
:107A4000882309F414CE80E00E945D11F2E09F2E9D
:107A500080E00E94010F882309F40FCE82E20E9489
:107A60005D11E3E09E2E8CE00E94170F882309F43D
:107A70000ACE8EE00E94951187E10E94170F88239D
:107A800009F407CE80E00E94951180E00E94170F54
:107A9000882309F404CE82E20E9495118EE00E94B0
:107AA000010F882309F401CE84E00E945D1174E087
:107AB000972E60E1A62E5FEEB52E8FE00E94010F9B
:107AC000882309F4F8CD83E00E945D1144E0942EF0
:107AD00030E2A32E2FEDB22E84E10E94010F882305
:107AE00009F4EFCD88E00E945D1194E0992E80E8C2
:107AF000A82E0FE7B02E85E10E94010F882309F41C
:107B0000E6CD81E00E945D1114E0912EB0E4AB2E31
:107B1000AFEBBA2E88E00E94010F882309F4DDCD77
:107B200084E20E945D11F4E09F2EEFE0AE2E70EF34
:107B3000B72E8EE00E94170F882309F4D4CD84E07D
:107B40000E9495118FE00E94170F882309F4D1CD70
:107B500083E00E94951184E10E94170F882309F4A5
:107B6000CECD88E00E94951185E10E94170F8823F1
:107B700009F4CBCD81E00E94951188E00E94170F97
:107B8000882309F4C8CD84E20E949511C4CD89E10F
:107B90000E945D11992444245CCD84E00E949511DB
:107BA0008FE00E94170F882309F40ECD83E00E9416
:107BB000951184E10E94170F882309F40BCD88E00A
:107BC0000E94951185E10E94170F882309F408CDC2
:107BD00081E00E94951188E00E94170F882309F424
:107BE00005CD84E20E94951101CD84E20E945D11D1
:107BF000992493942FE0A22E90EFB92ED9CC81E056
:107C00000E945D119924939440E4A42E3FEBB32E7F
:107C1000C9CC88E00E945D119924939460E8A62E57
:107C20005FE7B52EB9CC83E00E945D11992493944F
:107C3000E0E2AE2E7FEDB72EA9CC84E00E945D116C
:107C400099249394A0E1AA2EFFEEBF2E99CC8EE04A
:107C50000E9495118FCC8EE00E945D11992493941F
:107C6000AA24AA94BB2480CC81E00E94682572CE0D
:107C7000442009F02ECCE0CB442009F4DDCB9092D7
:107C80006204EE2089F0342D3E0DD60120E0822FD3
:107C9000830F6E2D0E945D41F301E90FF11D8D915F
:107CA00080832F5F2E1598F340910E06C30138CCC8
:107CB00083E00E94951184E10E94170F882309F444
:107CC0009ECD88E00E94951185E10E94170F8823C0
:107CD00009F49BCD81E00E94951188E00E94170F66
:107CE000882309F498CD84E20E94951194CD84E014
:107CF0000E94951178CD84E20E945D11A1E09A2A3C
:107D00001FE0A12EB0EFBB2E68CD81E00E945D1177
:107D100091E0992A80E4A82E0FEBB02E58CD88E090
:107D20000E945D1181E0982A20E8A22E9FE7B92EDB
:107D300048CD83E00E945D11F1E09F2A40E2A42E2D
:107D40003FEDB32E38CD84E00E945D11E1E09E2A24
:107D500060E1A62E5FEEB52E28CD8EE00E94951133
:107D60001ECD8EE00E945D11B1E09B2AAA24AA9448
:107D7000BB240FCD8CE00E945D11992402CD82E0DE
:107D80000E945D11409084054194992493946DCB99
:107D900080E20E945D1199244424FF2455245DCB88
:107DA0006091920681E141E10E945425AECD60913F
:107DB000920682E142E10E945425A1CD6091920693
:107DC00080E145E00E94542594CD609192068FE0B9
:107DD00044E00E94542587CD0E940C1282E20E944A
:107DE0005D1130926C0481E20E945D118091620409
:107DF000882309F48FC082E00E94791181E00E94FB
:107E000027026BCD8BE00E945D119924A5CBEE205B
:107E100009F43CCD860107C00F5F1F4F802F8C19DE
:107E20008E1508F033CD0E94E000F82EEFE3E8173E
:107E300098F30E94E000682D0E945D41F301E90F74
:107E4000F11DF0808F2D90E08F7090708D30910536
:107E5000B9F00E9791F09F2D9A21D8018C918B212A
:107E6000982B9C93D9CFF7EFFF2203CDE7EFFE22AB
:107E70008F2D90E08F709070F9CC87EFF822EBCFC8
:107E8000F7EFFF228F2D90E08F709070E2CF84E0AB
:107E90000E94682595CD82E00E9495118091AB06E5
:107EA0006091EC064091080620910E0602E516E06E
:107EB0000E941A2840910E06C801B6010E9471372F
:107EC000E82E1092620435CD8E2D869509F425CBCF
:107ED000D6016E2D6150262F281B8C91F601E60FDE
:107EE000F11D90819D93808361506217B1F715CB8E
:107EF00082E00E9495118091AB066091EC06409162
:107F0000080620910E0602E516E00E94CD27109289
:107F1000620405CD82E00E94951170CFF39481E058
:107F2000F8228DE00E949511FF2009F07BC0882483
:107F30000E946113C2CA82E00E94951159CD6091DE
:107F40000E0682E596E0A60126E835E00E94762539
:107F5000E82E882311F1860106C00F5F1F4F802F86
:107F60008C198E15D0F40E94E000F82EBFE3B817EC
:107F7000A0F30E94E000F80120816E2D0E945D4177
:107F8000F601E90FF11D8081D8018C9320830F5FEA
:107F90001F4F802F8C198E1530F360910E0682E5ED
:107FA00096E0A60126E835E00E94572640910E068D
:107FB00082E596E0B6010E947137AFCAEE2009F45F
:107FC000ACCA860107C00F5F1F4F802F8C198E151A
:107FD00008F0A3CA0E94E000F82E8FE38F1598F3F3
:107FE0000E94E000D8012C916E2D0E945D41F601A7
:107FF000E90FF11D80818A219B2D9223892B8C937F
:1080000080818B212A21822B8083DDCF8DE00E940D
:108010005D1188EC95E0B30140915C040E947137DA
:10802000882E53CC8DE00E945D1188EC95E0B30161
:1080300040915C040E947137882E40910E0682E5C3
:1080400096E0B6010E947137E82EA3E09A2E4424F0
:108050006FCF81E00E946825D3C9EF92FF920F9302
:108060001F930E94B0108091F906882309F421C162
:1080700084E00E946825FF24F39407C0113009F4BE
:1080800071C00E948E278823C9F00E94B010109101
:1080900092061330D9F0143088F31430E9F11D3012
:1080A00081F781E00E94002C809192068D3049F387
:1080B00010926C040E948E27882339F70E94702743
:1080C0000E94B01010919206133029F70E946E257D
:1080D000882309F092C00E94E026882321F01092A4
:1080E0005E0410926C040E94960F882309F072C0FF
:1080F0008091F906882329F686E10E94010F8823E2
:1081000009F0CCC086E10E94170F882309F4B9CF8B
:1081100080E00E94E318B5CF0E946E25882309F005
:1081200081C080E00E94002C0E945D278091920611
:10813000843011F010926C048091F906882309F4C0
:108140006DC080916B04813009F09BCF10926B045D
:108150000E94B324882309F494CF1F910F91FF90BC
:10816000EF9008950E946E25882309F077C080E083
:108170000E94002C86E10E94010F882301F586E110
:108180000E94170F8823B9F40E945D278091920600
:10819000813011F010926C048091F906813009F45D
:1081A00079C00E94B324882309F46BCF1F910F91EB
:1081B000FF90EF90089580E00E94E318E5CF80E003
:1081C0000E944C2590919A06890F60E040E00E9441
:1081D000CC18D5CF182F11500E944113812F0E9427
:1081E0001813109393068091F906882309F080CF25
:1081F0008091930680939A067BCF0E940C12F09296
:108200005E0481E00E94270284E20E945D11809159
:1082100093060E941813F0926C045DCF81E00E94D7
:1082200068258FCF0E940C1282E20E945D11F092AD
:108230006C0481E20E945D118091080660910E0637
:108240004091810520910F0600910806E0907F057E
:108250000E94531481E00E94270263CF0E940C12F7
:1082600082E20E945D1110936C0481E20E949511DC
:108270008091080660910E064091810520910F06BD
:1082800000910806E0907F050E94531481E00E944F
:1082900027026DCF84E00E94682583CF80E00E9492
:1082A0004C2590919A06890F60E040E00E94CC181E
:1082B00029CF81E00E946825DECE991B79E004C0B9
:1082C000991F961708F0961B881F7A95C9F7809515
:1082D0000895AA1BBB1B51E107C0AA1FBB1FA6170D
:1082E000B70710F0A61BB70B881F991F5A95A9F75F
:1082F00080959095BC01CD01089597FB092E072626
:108300000AD077FD04D0E5DF06D000201AF470957E
:1083100061957F4F0895F6F7909581959F4F089549
:10832000A1E21A2EAA1BBB1BFD010DC0AA1FBB1F79
:10833000EE1FFF1FA217B307E407F50720F0A21BEB
:10834000B30BE40BF50B661F771F881F991F1A9458
:1083500069F760957095809590959B01AC01BD0182
:08836000CF010895F894FFCF4E
:1083680001000100010001000100010001000100FD
:108378000100010001000100010001C0008000406F
:10838800007F20640F04050607111210130E040560
:108398000607111210130409050A06070B110C121F
:1083A8000D101325212326272422201D1E1B191FEB
:1083B8001C1A1012180F110C130E0B140D0A151697
:1083C80009170405080306010700020320191A18F3
:1083D8000C0B0A090420191A180C0B0A092221256A
:1083E8002320191A18241B1C0F0E0D04030A0C0B4A
:1083F8000908010200201B191C1A180F0C0E0B0D7E
:108408000A0926271D1E1F10121113141516170509
:1084180006076E306E783078000100070E091C1BC5
:108428001215383F363124232A2D70777E796C6BEC
:108438006265484F464154535A5DE0E7EEE9FCFB5C
:10844800F2F5D8DFD6D1C4C3CACD90979E998C8B4C
:108458008285A8AFA6A1B4B3BABDC7C0C9CEDBDCBC
:10846800D5D2FFF8F1F6E3E4EDEAB7B0B9BEABACAC
:10847800A5A28F88818693949D9A2720292E3B3C1C
:1084880035321F18111603040D0A5750595E4B4C0C
:1084980045426F68616673747D7A898E878095928C
:1084A8009B9CB1B6BFB8ADAAA3A4F9FEF7F0E5E26C
:1084B800EBECC1C6CFC8DDDAD3D4696E67607572DC
:1084C8007B7C51565F584D4A4344191E17100502CC
:1084D8000B0C21262F283D3A33344E49404752553C
:1084E8005C5B7671787F6A6D64633E39303722252C
:1084F8002C2B0601080F1A1D1413AEA9A0A7B2B59C
:10850800BCBB9691989F8A8D8483DED9D0D7C2C58B
:10851800CCCBE6E1E8EFFAFDF4F30409050A060717
:108528000B110C120D1013000100010001000100D5
:10853800010001000100010001000100010001002B
:1085480001C000800040000606011718191A1B1CFC
:108558001D1E1F202122233F3F3F0B0C0D0E0F1025
:10856800111213141516173F3F3F232425262728D9
:10857800292A2B2C2D2E2F3F3F3F1718191A1B1C69
:0C8588001D1E1F202122233F3F3F150035
:00000001FF
